:020000040000FA
:0600000075EF36F012005E
:0600080082EF32F012004D
:0600180090EF32F012002F
:06002A000300626D0000FE
:100030008000000068000000586D00006E0F000096
:100040000A000000526D0000FA03000006000000E4
:100050000101D86BD96B0301326B00018F6B120069
:10006000A4EC10F0DF6A00019051020A59E0030A83
:100070001CE0010A65E194EC2AF0000963E10E013D
:100080005D5160E05D51E66EE66A5E0EE66E0E0E54
:10009000E66E06EC2BF0E8EC0EF00001010E906F1E
:1000A000D7DF0E01640E3E6F4DD098EC2AF00009A8
:1000B00033E00001020E906F0E015D29156AE850D1
:1000C00000018D5F15508E5B0E015D51146E156A37
:1000D000960ED8801456000E15561406155A14C0E4
:1000E000E6FF15C0E6FF5D51176A5D0F166E0E0E36
:1000F0001722010E1626000E172216C0E6FF17C0A3
:10010000E6FF5D0EE66E0E0EE66EAEEC2BF0186EA0
:10011000060EE15E185016D00E013E5113E110D0CC
:100120000101D8510AE0D8C1D9F1D851020802E240
:100130000E015D6B0001906B05D00E013E5102E196
:10014000010EDF6EDF5008E00101D9690E015D6B21
:100150000001906B33EC2BF0E552CCEF0EF094ECF9
:100160002AF0000906E10001905103E10E015D5102
:1001700001E0010C000CD0EC0EF0FC0EDB50000195
:10018000156A8D25146E8E511522010E1426000E4F
:100190001522F30E145C0E0E15581CE2FC0EDB50FB
:1001A00052EC11F0EF6EFC0EDBCFE6FFE66AFAECE4
:1001B0000EF0010E2DEC10F083EC2BF0166E060EF7
:1001C000E15E1650FC0EDB28146E156AE850E4EC74
:1001D0000FF001D0010ECCEF0EF0D0EC0EF0020EBD
:1001E0000001176A8D25166E8E51172216C0E6FF84
:1001F00017C0E6FFFAEC0EF034EC2CF031EC11F005
:10020000E7CF17F0E552E7CF16F01650F324146E3F
:100210001750F420156EF30E145C0E0E15581BE2E9
:1002200035EC11F0010EF32452EC11F0EF6EFAEC04
:100230000EF0010E00012DEC10F0FAEC2BF0E8ECC2
:100240000EF035EC11F0020E1426000E152214509B
:10025000E4EC0FF001D0010ECCEF0EF0D0EC0EF07C
:100260000101C651040A49E0050A02E0030A43E11C
:10027000D85141E198EC2AF000093DE000018F518E
:1002800007E1FE0EDB50FE0803E00101E26B33D014
:1002900053EC10F009E2ECEC0FF0020E8F5D07E179
:1002A000FE0EDB50FE0803E00101D86924D00101F5
:1002B000E25102E1010EE26FFE0EDB50FD0869E142
:1002C000020E00018F5DEA6A320FE96E030EEA2228
:1002D000EF50FF0A0AE0050A05E0010A09E1010101
:1002E000010E08D00101040E05D00101050E02D057
:1002F0000101020ED86F000E4DD0D85148E198ECA4
:100300002AF0000944E0FE0EDB502E0803E1010153
:10031000010E08D00101E20507E1FE0EDB500D08D9
:1003200003E1020EE26F35D0020EE25D0EE1FE0E39
:10033000DB500A080AE1E26B00018F5103E0010182
:10034000020E18D00101010E15D079EC10F0CFEC9F
:1003500017F018EC10F0F350F4100EE179EC10F0F7
:10036000E1EC17F0E552E552F350F41005E101011C
:10037000E26B040ED86F0DD0000153EC10F004E3D3
:100380000101E26BD86905D0ECEC0FF002D001015D
:10039000E26B000ECCEF0EF038EC2BF015EC2BF0EE
:1003A0005FDE0101D95112000E013E5102E1640EDF
:1003B0003E6F0E013E5103E0EFDF0009FAE001015C
:1003C000D95105E10E013E5102E10101D969010156
:1003D000D951020802E2D9511200000CA4EC10F02D
:1003E0000101C60503E0020EC65D04E1DF6A010EED
:1003F000D96F45D0FE0EDBCFC6F1D2EC29F0FE0E50
:10040000DB50020A19E0030A36E10001FE0EE16F3B
:10041000E26F580EE36FE00EE46F800EE66E250E7D
:10042000CAEC10F05FEC10F003E11C0E94EC10F03D
:10043000DF5025E1E66A1BD00001FE0EE16FE26F9E
:10044000280EE36FE00EE46FB00EE66E040ECAEC09
:1004500010F05FEC10F007E1100EE66E270EE66E6E
:10046000E66A5CEC11F0DF500AE1010EE66E37EC53
:1004700007F0E55203D0050E0101D96FDF6EDF50A2
:1004800002E00101C66BDF50E552CCEF0EF0A4ECA8
:1004900010F0DF6AF80EDB50DF5C38E2F90EDBCFDC
:1004A00006F0FA0EDBCF07F0FB0EDBCF08F0FC0EF8
:1004B000DBCF09F00A0E0B6E0C6A0D6A0E6A04ECB3
:1004C00036F00250E66E4AEC0FF0E552E750EF6E60
:1004D000FFEC0EF0B6EC0FF00A0E0B6E0C6A18EC87
:1004E0000FF004EC36F078EC0FF0040ED8901436D0
:1004F000153616361736E806F9E14AEC0FF01450B7
:10050000EF26FFEC0EF0020EDF26C4D7E552CCEF4B
:100510000EF006EC11F0DE6ADE6ADE6ADD6ADD529C
:10052000DD52FC0EDB5010E0FC0EDB06EBEC0EF0B7
:10053000EF380F0BA4EC0FF0DD52DD52EBEC0EF0B8
:10054000EF50A4EC0FF0EBD7F7EC0FF0050EE15CE9
:1005500002E2E16AE552E16ECCEF0EF00AEC11F036
:10056000050EE76F0A0EE66E91EC10F065EC10F0E8
:10057000146E070EE15E14500101FD0EED6F0B0EBF
:10058000C2EC0EF0CCEF0EF00AEC11F0060EE76FA5
:10059000FE0EDB50030A0FE0010A0BE0030A07E03E
:1005A000010A03E0030ED96F0AD0050E05D0020E32
:1005B00003D0E86B02D0010EE86F01EC11F0CCEF34
:1005C0000EF00AEC11F00D0EE76FE150FD0FD5ECC7
:1005D00010F00F0ED880EE54270EED5403E2030EF8
:1005E000D96F1FD0080EE66E1FEC10F0166A176A5E
:1005F0000A0E0B6E0C6A3AEC11F002C0E6FF03C063
:10060000E6FF04C0E6FF05C0E6FF65EC10F0186EDB
:10061000070EE15E18500101FD0EEC6F0A0EC2ECF0
:100620000EF0CCEF0EF0A4EC10F0DEEC0EF00F0E9E
:10063000E76FDF6AFE0EDB50050A14E0070A0FE0E1
:10064000060A0DE0050A09E0020A07E0030A03E0D2
:10065000030ED96F0DD0100E03D0110E01D0120E63
:10066000E86F04D0010ED96F000E02D001EC11F03A
:10067000E552CCEF0EF0DEEC0EF0080E9BEF10F022
:100680000AEC11F0080EE76F1FEC10F00A0E0D6E69
:100690000E6A14C008F015C009F05FEC36F004C013
:1006A00014F005C015F03FEC11F00A0E0D6E0E6A45
:1006B00016C008F017C009F05FEC36F008C016F05D
:1006C00009C017F00A0E0D6E0E6A5FEC36F004C01A
:1006D00016F005C017F0040ED89016361736E80449
:1006E000FBE1145016240101E86F01EC11F0CCEF8E
:1006F0000EF0DEEC0EF0070E9BEF10F0DEEC0EF0CD
:10070000090E9BEF10F0DEEC0EF00A0E9BEF10F0DE
:10071000A4EC10F0DEEC0EF0030E9BEC10F0DF6E9C
:10072000DF5022E1020E0101D95D1CE1030E03013D
:10073000365D18E1050EE66E370EE66E030EE66EC8
:10074000E8DE31EC11F006C0CBF107C0CCF108C0F7
:10075000CDF109C0CEF10EEC0FF046EC11F01EEC1D
:1007600011F002D0030EDF6EDF50E552CCEF0EF039
:10077000DEEC0EF06BEC10F0010EE96F080EC2EF2C
:100780000EF0DEEC0EF06BEC10F0E96B080EC2EF31
:100790000EF0A4EC10F0030E0101C65D04E1DF6A67
:1007A000010ED96F25D0030EC66FE9EC29F0949C99
:1007B0009694949E0001E551E8B0828EE8A0829E56
:1007C000E651E8B08484E8A08494E751E8B0828CD4
:1007D000E8A0829C01012B0EFA6F020EF96F580EF1
:1007E00094EC10F0DF5004E1E66A41DBE552DF6E85
:1007F000DF50E552CCEF0EF0D9CFE6FFE1CFD9FFC5
:10080000020EE1263F0E0101FA170001E55107E053
:100810000101FA1DE76E010EE7CFDBFF03D0010EE9
:10082000FAC1DBFF010EDF6EDF5014E0010EDB507A
:10083000DF1402E0828E01D0829E0001E65104E0C6
:1008400084940000848403D0848400008494DF9E18
:10085000DF46EAD70001E55107E00101F91DE76E27
:10086000010EE7CFDBFF03D0010EF9C1DBFF010E64
:10087000DF6EDFB614D0010EDB50DF1402E0828E93
:1008800001D0829E0001E65104E08494000084843B
:1008900003D0848400008494DF9EDF46EAD7000101
:1008A000E55107E00101F71DE76E010EE7CFDBFF21
:1008B00003D0010EF7C1DBFF080EDF6EDF5014E03E
:1008C000010EDB50DF1402E0828E01D0829E000117
:1008D000E65104E084940000848403D08484000002
:1008E0008494DF9EDF46EAD70001E55107E001016D
:1008F000F81DE76E010EE7CFDBFF03D0010EF8C154
:10090000DBFF010EDF6EDF5014E0010EDB50DF1461
:1009100002E0828E01D0829E0001E65104E08494C0
:100920000000848403D0848400008494DF9EDF462A
:10093000EAD70001E75104E0829C0000828C03D0DA
:10094000828C0000829C000E00D0146E020EE15CCE
:1009500002E2E16AE552E16E1450E552E7CFD9FFB9
:100960001200D0EC0EF0030EE126060EE66EC3EC8C
:100970000FF057EC11F018EC0FF004EC36F006C055
:1009800014F007C015F008C016F009C017F006C033
:10099000E6FF07C0E6FF08C0E6FF09C0E6FFDAECA5
:1009A00010F075DD186E070EE15E1850010EDBCFFA
:1009B000F8F1F00EDF140101F76F0F0EDF14146E63
:1009C000050E145C01E3F7879CEC0FF0000E146E2B
:1009D000030EE15C02E2E16AE552E16E1450CCEFF5
:1009E0000EF0D9CFE6FF000ECCEF0EF0D9CFE6FF28
:1009F000000ECCEF0EF00DEC11F00DE0210E26EC08
:100A000010F009E2FE0EDB041F0B0101FA6F9CECF3
:100A10000FF0000E03D00101030ED96FCCEF0EF0E2
:100A20000101FA9B9CEC0FF0000C0101FA8B9CEC8D
:100A30000FF0000C0DEC11F0020805E2020EF36E4F
:100A4000FE0EF3CFDBFFFE0EDBCFF9F19CEC0FF0D7
:100A5000000ECCEF0EF00DEC11F004E11EEC11F0E5
:100A6000000E03D00101030ED96FCCEF0EF0A4EC01
:100A700010F0040E0101C65D04E1DF6A010ED96FBA
:100A800017D0040EC66FD2EC29F0E66A4B0ECAEC02
:100A900010F09D889D8A1C0E94EC10F0DF5004E14C
:100AA000E66AD4EC0DF0E552DF5002E00101C66BBE
:100AB000DF50E552CCEF0EF0D0EC0EF00E0EE1263A
:100AC000ADEC10F0B10EEE54080EEE54190EEE54CB
:100AD00007E2DE6AB10EDE6E080EDE6E190E17D06A
:100AE000ADEC10F03B0EEE54580EEE54080EEE54E2
:100AF00007E2DE6A3B0EDE6E580EDE6E080E07D091
:100B0000800EDE6EBA0EDE6E8C0EDE6E010EDD6EB7
:100B1000DD52DD52CBEC0FF0D9CFE9FF4EEC0FF0F8
:100B2000FB0E14C0DBFFFC0E15C0DBFFFD0E16C074
:100B3000DBFFFE0E17C0DBFF91EC10F0880EE66EB7
:100B40006C0EE66E000E22EC11F0E15E14503AECF1
:100B50000FF0A7EC10F0E76E0D0EE7CFDBFFDB50D8
:100B600054E1020E0101D95D50E100018F514DE0C9
:100B70005D0EE66E320EE66E030EE66EBBEC2CF0FA
:100B800031EC11F00B0EF3CFDBFF0C0EF4CFDBFFDB
:100B9000F3CF14F0F4CF15F0F350F41006E00B0E81
:100BA000DB2A0C0E0BE3DB2A09D0D9500B0FE96EC0
:100BB000DACFEAFF320EEE6E030EED6E0B0EDBCFD8
:100BC000E6FF0C0EDBCFE6FF2DEC31F0E552E552EF
:100BD000FB0E06C0DBFFFC0E07C0DBFFFD0E08C0EE
:100BE000DBFFFE0E09C0DBFFC3EC0FF011EC11F0D0
:100BF000EE5014240101CB6FEE501520CC6FEE5057
:100C00001620CD6FEE501720CE6F0D0EDB50146EF8
:100C10000E0EE15C02E2E16AE552E16E1450CCEFA7
:100C20000EF0D0EC0EF00E0EE126FE0EDB50030AA5
:100C300021E0070A1FE0060A10E0030A08E0010AA3
:100C400063E1850EE66E6C0EE66E000E0BD0820E32
:100C5000E66E6C0EE66E000E05D07F0EE66E6C0E34
:100C6000E66E000EE66E3AEC0FF01BEC2CF0146E04
:100C7000050E48D0D880000E0101CF55B10ED055D9
:100C8000080ED155190ED25508E281EC0FF0B10EC5
:100C9000155E080E165A190E11D0D880000ECF55C9
:100CA0003B0ED055580ED155080ED2550CE281ECB2
:100CB0000FF03B0E155E580E165A080E175A14C048
:100CC000DFFF010E0CD081EC0FF0800E145EBA0E27
:100CD000155A8C0E165A010E175A14C0DFFF15C094
:100CE000DBFF020E16C0DBFF030E17C0DBFF11ECAB
:100CF00011F0D5EC0EF0770EE66E6C0EE66E000E7F
:100D000022EC11F0E15E14503AEC0FF0A7EC10F079
:100D1000146E0E0EE15C02E2E16AE552E16E1450DF
:100D2000CCEF0EF0D0EC0EF0030E0101D35D03E02A
:100D3000040ED35D04E17EEC10F0E55201D0000E0C
:100D4000CCEF0EF016EC11F0240E26EC10F011E2B0
:100D500079EC10F0720EE66E6C0EE66E000EE66E2A
:100D6000DAEC10F0E5EC34F0146E070E61EC11F0E3
:100D700003D00101030ED96F146E040EE15C02E290
:100D8000E16AE552E16E1450CCEF0EF01EEC11F06A
:100D9000000C16EC11F06E0EE66E6C0EE66E000E98
:100DA0001CEC0FF002E2E16AE552E16E1450CCEF68
:100DB0000EF016EC11F0FE0EDB50000806E26B0E92
:100DC000E66E6C0EE66E000E05D0680EE66E6C0EDA
:100DD000E66E000E1CEC0FF002E2E16AE552E16EF5
:100DE0001450CCEF0EF00DEC11F004E11EEC11F0FC
:100DF000000E03D00101030ED96FCCEF0EF0D2EC40
:100E000029F01EEC11F0C66B000CD2EC29F01EECA0
:100E100011F000018B6B0101630EC66F000CA4EC96
:100E200010F0FE0EDB50630A16E0670A12E0070AB4
:100E30000EE0020A06E0030A04E0020A0FE1DFDF27
:100E40000BD0EEEC10F0EEEC01F0E55205D0A1DC99
:100E500003D00DDE01D0D9DFDF6E05D0030EDF6ECB
:100E60000101D96FC66BDF50E552CCEF0EF066EC96
:100E700011F01CE0670A14E0070A0EE0020A07E01E
:100E8000030A05E0020A15E146EC0FF014D0EEEC7F
:100E900010F0C4EC02F007D0EEEC10F0DCDD03D073
:100EA000EEEC10F0A0DFE552DF6E05D0A0EC0FF005
:100EB00002D0DF68D969DF50E552CCEF0EF006ECC6
:100EC00011F0FD0EDBCF06F0FE0EDBCF07F0086A57
:100ED000096A400E0B6E420E0C6E0F0E0D6E27EC63
:100EE0000FF00DE0030A0BE0010A09E0070A07E032
:100EF000670A05E0630A06E146EC0FF005D087ECCF
:100F000010F002D0DF68D96982EC10F002E2E16AE9
:100F1000E552E16E1450CCEF0EF006EC11F0FB0E32
:100F2000DBCF06F0FC0EDBCF07F0FD0EDBCF08F0C9
:100F3000FE0EDBCF09F057EC11F00D6A27EC0FF035
:100F40000DE0030A0BE0010A09E0070A07E0670A5F
:100F500005E0630A06E146EC0FF005D087EC10F0DF
:100F600002D0DF68D96982EC10F002E2E16AE55252
:100F7000E16E1450CCEF0EF006EC11F01FEC10F007
:100F8000166A176A57EC11F03AEC11F0C70EE96EC9
:100F9000010EEA6E8AEC0FF0010E14C0DBFF020EA8
:100FA00015C0DBFF030E16C0DBFF040E17C0DBFF0E
:100FB0000101C651010A0DE0030A0BE0010A09E034
:100FC000070A07E0670A05E0630A06E146EC0FF04E
:100FD00005D087EC10F002D0DF68D96982EC10F000
:100FE00002E2E16AE552E16E1450CCEF0EF0D0EC73
:100FF0000EF0070EE126020EDB68010EF36E030E03
:10100000F3CFDBFF040EDB6A050EDB6A060EDB6A3C
:10101000DF6ADFCF14F0156A166A030ED890143613
:1010200015361636E806FAE1D8EC0FF01424F36E04
:10103000EE501520F46EEE5016200DEC10F0090065
:10104000F5500900F5100900F5100800F51001E150
:1010500091D0F40EDBCF14F0F50EDBCF15F0F60EC9
:10106000DBCF16F0F70EDBCF17F0DFCF18F0196AE1
:101070001A6A030ED890183619361A36E806FAE1BD
:10108000D8EC0FF01824F36EEE501920F46EEE50E9
:101090001A20F86EF4CFF7FFF3CFF6FF0900F550F2
:1010A000145C0900F55015580900F5501658090050
:1010B000F55017585DE3F40EDBCF1BF0F50EDBCFD8
:1010C0001CF0F60EDBCF1DF0F70EDBCF1EF0DFCFEE
:1010D0001FF0206A216A030ED8901F362036213671
:1010E000E806FAE1D8EC0FF01F24F36EEE50202052
:1010F000F46EEE5021200DEC10F01B500900F55C51
:101100001C500900F5581D500900F5581E500900E3
:10111000F5582EE3030EDBCF22F0040EDBCF23F0D5
:10112000050EDBCF24F0060EDBCF25F0D950F80FEB
:10113000D5EC10F0EE502216EE502316EE50241689
:10114000EE502516225023102410251011E0020E17
:10115000DFCFDBFFD950030FE96EDACFEAFFD8907B
:10116000EF36010EEB36020EEB36030EEB3602D0F5
:10117000DF2A4FD7020EDB50146E070EE15C02E24D
:10118000E16AE552E16E1450CCEF0EF0D0EC0EF0B7
:10119000020EE126010EDB68DF6A5DEC0FF0EECF98
:1011A00014F0EECF15F0EECF16F0EFCF17F014508D
:1011B00015101610171017E0B6EC0FF05DEC0FF0DD
:1011C0001450EE180EE11550EE180BE11650EE1803
:1011D00008E11750EE1805E104E1010EDFCFDBFF57
:1011E00002D0DF2ADAD7010EDB50146E020EE15C6A
:1011F00002E2E16AE552E16E1450CCEF0EF0A4EC8D
:1012000010F0DF6A91EC10F083C0E6FF84C0E6FFC7
:1012100085C0E6FF86C0E6FF940EE66E5E0EE66EC3
:10122000000EDDEC0FF005E1000E151802E1000ED6
:10123000DF8091EC10F087C0E6FF88C0E6FF89C030
:10124000E6FF8AC0E6FF940EE66E5F0EE66E000EC5
:10125000DDEC0FF002E1000E151801E0DF8291ECE9
:1012600010F0910EE66E000EE66E90DF166E060E22
:101270004BEC11F002E1000E151801E0DF84DF50A5
:10128000E552CCEF0EF016EC11F0BEEC0EF037ECA0
:1012900010F011E3E3EC10F0A00EEE542F0EEE541C
:1012A000C50EEE54010EEE5406E3A00EDE6E860E61
:1012B000DE6E010E97D0BEEC0EF0C00EEE5C320E6C
:1012C000EE580A0EEE58030EEE581BE3E3EC10F056
:1012D000800EEE54F90EEE54370EEE54030EEE541B
:1012E00010E3040E0101C65D06E0200EDE6EA10EC5
:1012F000DE6E070E77D0400EDE6E420EDE6E0F0EF3
:1013000071D0D1EC10F0440EEE58950EB2EC0FF007
:101310000FE3ADEC10F04D0EEE54D20EEE54080E6D
:10132000EE5406E3C00EDE6E270EDE6E090E5AD0B6
:10133000DFEC10F0730EEE583B0EEE580D0EEE582B
:1013400010E3E3EC10F0400EEE543A0EEE54690E4A
:10135000EE540D0EEE5405E3DE6A6A0EDE6E180ED4
:1013600041D0D1EC10F0B10EB2EC0FF0190EEE58E6
:1013700011E3E3EC10F0800EEE54740EEE54D20E36
:10138000EE541A0EEE5406E3400EDE6E4B0EDE6E89
:101390004C0E28D0DFEC10F06D0EEE58C30EEE5858
:1013A000350EEE5809E3ADEC10F0280EEE54500E59
:1013B000EE54370EEE5412E2D1EC10F0E60EEE5879
:1013C000E80EEE58490EEE580FE3ADEC10F06D0E3E
:1013D000EE547C0EEE544D0EEE5406E3DE6A1B0E08
:1013E000DE6EB70EDE6E03D0DE6ADE6ADE6ADD6AAE
:1013F000DD52DD52F7EC0FF0040EE15C02E2E16A2F
:10140000E552E16ECCEF0EF0A4EC10F0BEEC0EF065
:1014100037EC10F00AE3D1EC10F0A90EEE58C30E31
:10142000EE58010EEE5801E2E7D0ADEC10F0A90E37
:10143000EE54C30EEE54010EEE540CE2BEEC0EF070
:10144000A00EEE5C2F0EEE58C50EEE58010EEE58B3
:1014500001E203D1BEEC0EF0F00EEE5C180EEE5879
:101460000D0EEE58030EEE580CE3E3EC10F0D00E28
:10147000EE54AC0EEE54110EEE54030EEE5401E396
:10148000BBD0BEEC0EF0500EEE5C380EEE581A0ECD
:10149000EE58030EEE580CE3E3EC10F0100EEE5491
:1014A000EF0EEE54200EEE54030EEE5401E3A4D0E2
:1014B000BEEC0EF0700EEE5C2C0EEE58290EEE58BF
:1014C000030EEE580CE3E3EC10F0500EEE54310E28
:1014D000EE54300EEE54030EEE5401E38DD0BEEC0C
:1014E0000EF0E00EEE5C0C0EEE58A60EB2EC0FF015
:1014F0000BE3BEEC0EF0600EEE5C270EEE58AC0E69
:10150000B2EC0FF001E2A9D01AEC11F0F00EEE5897
:10151000BC0EB2EC0FF004E3E6EC10F001E29DD05B
:10152000DFEC10F0320EEE58CC0EB2EC0FF009E307
:10153000D1EC10F04D0EEE58D20EB2EC0FF001E2ED
:101540008CD0DFEC10F0C80EEE58B30EB2EC0FF0FA
:1015500008E3D1EC10F0E30EEE58B90EB2EC0FF048
:101560004BE3E6EC10F008E31AEC11F0250EEE5810
:10157000C90EB2EC0FF040E3E3EC10F0600EEE5455
:10158000710EEE54580EEE540D0EEE5409E21AECA4
:1015900011F03A0EEE58690EEE580D0EEE585DE35E
:1015A000ADEC10F0DE0EEE54390EEE541A0EEE5481
:1015B00026E21AEC11F0290EEE58860EEE581A0E9D
:1015C000EE581DE2DBDB400EEE1808E1200EEE18AF
:1015D00005E1490EEE1802E11A0EEE1810E0CEDB1E
:1015E000600EEE1808E1C10EEE1805E1500EEE187F
:1015F00002E11A0EEE1803E0010EDF6E31D0E3ECCB
:1016000010F0400EEE54290EEE54860EEE541A0ED3
:10161000EE5425E2DFEC10F0740EEE58D20EEE58C8
:101620001A0EEE581CE2AADB800EEE1808E16B0ED3
:10163000EE1805E1950EEE1802E11A0EEE180FE015
:101640009DDBA00EEE1808E10C0EEE1805E19D0ED4
:10165000EE1802E11A0EEE1802E0DF6801D0DF6A30
:10166000DF50E55299D39CDB090EE12691EC10F096
:101670000ADEAEDB010E06C0DBFF020E07C0DBFF99
:10168000030E08C0DBFF040E09C0DBFF91EC10F075
:10169000BBDE69EC11F0DFCF14F0000EE76E14181A
:1016A000E8AE02D0143403D0E750D880145410E2CE
:1016B000010EDBCF14F0020EDBCF15F0030EDBCFF3
:1016C00016F0040EDBCF17F059DB8AEC0FF00AD0CE
:1016D000DFCF14F0143413E3CBEC0FF0D950010F2B
:1016E000E96EDCDB050E14C0DBFF060E15C0DBFF68
:1016F000070E16C0DBFF080E17C0DBFF0DD03EDB68
:10170000050EEECFDBFF060EEECFDBFF070EEECFB2
:10171000DBFF080EEECFDBFF050EDBCF14F0060E6D
:10172000DBCF15F0070EDBCF16F0080EDBCF17F07E
:10173000F2EC10F0090EE15C02E2E16AE552E16EC2
:101740002BD32EDB080EE12600018C5103E00101B2
:10175000050ED36F0101D351050A56E0010A3CE0A2
:10176000070A27E0010A16E0030A06E0010A01E081
:101770007BD040EC10F078D0FBEC10F0EE50010183
:10178000CB5D146EEE50CC59156EEE50CD59166EE1
:10179000EE501FD0FBEC10F00101CB51EE24146E83
:1017A000CC51EE20156ECD51EE20166ECE51EE20AE
:1017B00011D080C018F081C019F01A6A1B6A185045
:1017C000CB5D146E1950CC59156E1A50CD59166E4A
:1017D0001B50CE59176E0BD080C014F081C015F08D
:1017E000166A176ACB0EE96E010EEA6E93DB040EE1
:1017F00014C0DBFF050E15C0DBFF060E16C0DBFFB5
:10180000070E17C0DBFF30D08EDB2DDFE1DA040ED0
:1018100006C0DBFF050E07C0DBFF060E08C0DBFFBE
:10182000070E09C0DBFF49EC10F0EE500101CB19A7
:101830000CE1EE50CC1909E1EE50CD1906E1EE5065
:10184000CE1903E102E1D36B0FD049EC10F0EE505A
:10185000CB5DEE50CC59EE50CD59EE50CE5902E250
:10186000020E01D0010ED36F49EC10F09EDAC7DCF6
:10187000AFDA146E0F0E00018215141407E0010E8A
:101880008B6F40EC10F00101D36B0DD08B6B040E0D
:10189000DBCFCFF1050EDBCFD0F1060EDBCFD1F1E0
:1018A000070EDBCFD2F1080EE15C02E2E16AE552FD
:1018B000E16E72D275DA160EE1260001825102E164
:1018C000DF6A10D091EC10F09ADC82DAE76E010E3C
:1018D000E7CFDBFFDBCFE6FF000182390F0BE552DC
:1018E000E714DF6EDF5008E1010EDBCFE6FF0F0EDD
:1018F0008215E552E7148B6FDF5004E0030EDF6EB4
:101900000101D96FDF5001E0A1D0020EC7C1DBFF9A
:10191000030EC8C1DBFF040EC9C1DBFF050ECAC13F
:10192000DBFF060ECBC1DBFF070ECCC1DBFF080ED1
:10193000CDC1DBFF090ECEC1DBFF0A0ECFC1DBFF3D
:101940000B0ED0C1DBFF0C0ED1C1DBFF0D0ED2C1DF
:10195000DBFFFB0EDBCFC7F1FC0EDBCFC8F1FD0ECA
:10196000DBCFC9F1FE0EDBCFCAF129EC11F0C7C104
:1019700006F0C8C107F0C9C108F0CAC109F046ECB9
:1019800011F0FB0EDBCFCBF1FC0EDBCFCCF1FD0E6B
:10199000DBCFCDF1FE0EDBCFCEF1D3DE8CDB2CE046
:1019A000670A1FE0070A17E0020A06E0030A04E0DC
:1019B000020A24E16BDA24D0B4DBAEEC02F069EC6D
:1019C00011F0DF501DE100018C511AE1D3C1E6FF97
:1019D00013EC03F00ED0A5DBB1EC04F031EC11F008
:1019E00008D09FDB5CEC05F069EC11F0DF5008E1FA
:1019F00085DBE552DF6E04D0A3DA02D0DF68D96957
:101A0000DF5024E0020EDBCFC7F1030EDBCFC8F1BD
:101A1000040EDBCFC9F1050EDBCFCAF1060EDBCF1A
:101A2000CBF1070EDBCFCCF1080EDBCFCDF1090EE9
:101A3000DBCFCEF10A0EDBCFCFF10B0EDBCFD0F137
:101A40000C0EDBCFD1F10D0EDBCFD2F1DF50146ED7
:101A5000160EE15C02E2E16AE552E16E14509CD19F
:101A6000D9CFE6FF020E98D16FDB060EEFDA25E242
:101A7000FE0EDBCFD3F165DE1EDB1DE0670A17E04B
:101A8000070A10E0020A0AE0030A08E0020A03E07B
:101A9000DF68D96916D0050EDF6E12D09FDB13EC1C
:101AA00003F006D0D3C1E6FFF6EC04F001D026DB4C
:101AB000E552DF6E06D044DA04D0030EDF6E01017A
:101AC000D96FDF50E55268D13FDBFD0EDBCF80F0F0
:101AD000FE0EDBCF81F0EFDA1BE0670A12E0070AA7
:101AE0000CE0020A06E0030A04E0020A13E1CED980
:101AF00013D080D9E1EC02F007D07CD9F1EC04F0EE
:101B000003D078D992EC06F0E552E552DF6E04D0AE
:101B100017DA02D0DF68D969DF50E5523DD111DB19
:101B20000EE0030A0CE0010A0AE0070A08E0670A6F
:101B300004E0630A04E1AAD904D002DA02D0DF6823
:101B4000D969DF50E55228D1FCDA0EE0030A0CE037
:101B5000010A0AE0070A08E0670A04E0630A04E1F0
:101B600095D904D0EDD902D0DF68D969DF50E552AC
:101B700013D10101C6510BE0020ED96FCBC1DAF1CE
:101B8000CCC1DBF1CDC1DCF1CEC1DDF1000C050C27
:101B90000101C65108E0020ED96FD3C1DAF1DB6B47
:101BA000DC6BDD6B000C050CCCDA12E0030A10E0F4
:101BB000010A08E0600A04E0630A0AE167D90AD072
:101BC000BFD908D00BDBFBEC04F0E552DF6E02D08E
:101BD000DF68D969DF50E552DFD078DB11E0620AB7
:101BE0000BE0030A09E0010A04E0030A0CE14ED904
:101BF0000AD010EC05F002D0B8EC03F0DF6E03D091
:101C0000010ED96FDF6ADF50E552C6D05FDB11E00D
:101C1000620A0BE0030A09E0010A04E0030A0CE18E
:101C200035D90AD015EC05F002D0C1EC03F0DF6E17
:101C300003D0010ED96FDF6ADF50E552ADD081DAF3
:101C400012E0030A10E0010A08E0600A04E0630AF7
:101C50000AE11CD90AD074D908D0C0DA1AEC05F010
:101C6000E552DF6E02D0DF68D969DF50E55294D0CB
:101C700068DA0CE0030A0AE0010A1CE0600A04E0EA
:101C8000630A18E103D918D05BD916D0B3D82ADA81
:101C900003E183EC03F0DF6EDF5003E188EC03F037
:101CA000DF6EDF5003E100018B6B06D00001010EF7
:101CB0008B6F02D0DF68D969DF50E5526DD041DA11
:101CC0000CE0030A0AE0010A0FE0600A04E0630A7C
:101CD0000BE1DCD80BD034D909D08CD803DA06E17B
:101CE0007EEC03F0DF6E02D0DF68D969DF50E55289
:101CF00053D027DA0CE0030A0AE0010A0CE0600A7C
:101D000004E0630A08E1C2D808D01AD906D088ECEA
:101D100003F0DF6E02D0DF68D969DF50E5523CD0B6
:101D200010DA0CE0030A0AE0010A0CE0600A04E0A1
:101D3000630A08E1ABD808D003D906D079EC03F0E8
:101D4000DF6E02D0DF68D969DF50E55225D0F9D9BE
:101D50000CE0030A0AE0010A0CE0600A04E0630AEE
:101D600008E194D808D0ECD806D03BEC03F0DF6E45
:101D700002D0DF68D969DF50E5520ED0D950FB0F91
:101D8000D5EF10F0E66EE30EE66E010EE66EBBECEC
:101D900000F067DAD4EF01F0E552E7CFD9FF120087
:101DA000D9CFE6FFE1CFD9FF1200EECFE6FFEECFAD
:101DB000E6FFEECFE6FFEFCFE6FF1200E1C0E3F172
:101DC000E2C0E4F1E3C0E5F1E4C0E6F10101120094
:101DD00048DAE552120025DAC3D9CCEC35F005C05B
:101DE000EDFF04C0EDFF03C0EDFF02C0EFFFFC0EEE
:101DF000DB50C4D1FD0EDBCFE6FFEEEF10F0D95083
:101E0000F90FD3D9ADD904EC36F009C0EDFF08C005
:101E1000EDFF07C0EDFF06C0EFFF120006C0C7F1DF
:101E200007C0C8F108C0C9F109C0CAF129EF11F013
:101E30000D6A0E6AF2EF10F0E66EBCD91BEC2CF0C6
:101E4000146E050E3EDA146E040EE15C12000E6A8A
:101E5000CCEC35F0010E02C0DBFF020E03C0DBFF4D
:101E6000030E04C0DBFF040E05C0DBFF0101C651F9
:101E7000010A1200D950040FE66E000EDA20E66E59
:101E80001200E6520101C651010A1200050EDF6E72
:101E9000D96F1200DF50FE0BE84270D1DACFEAFFB3
:101EA000EE50185C146EEE501958156EEE501A581C
:101EB000166EEE501B58176E1200FD0EDBCF18F099
:101EC000FE0EDBCF19F0DF50040D1850F324E96E3D
:101ED0001950F420EA6E120006C0DEFF07C0DEFFD4
:101EE00008C0DEFF09C0DDFFDD52DD5211EF11F049
:101EF00002C014F003C015F004C016F005C017F0BE
:101F00001200CFC114F0D0C115F0D1C116F0D2C16A
:101F100017F01200EE501426EE501522EE50162245
:101F2000EE5017221200CBC1E6FFCCC1E6FFCDC1B7
:101F3000E6FFCEC1E6FF1200FCEC03F01EEF11F04D
:101F4000010ED96FDF6A12000F0B146E156A166A44
:101F5000176AE850DE261550DE221650DE22175092
:101F6000DD221200EE58080EEE581200F90EDBCFFB
:101F700014F0FA0EDBCF15F0FB0EDBCF16F0FC0EE3
:101F8000DBCF17F01200FB0EDBCF14F0FC0EDBCF23
:101F900015F03FEF11F0FB0EDBCF18F0FC0EDBCF9E
:101FA00019F0FD0EDBCF1AF0FE0EDBCF1BF0120096
:101FB000D950FC0FFAD8EE501200E66EF7EC07F09D
:101FC000166E0B0E4BEF11F000018D2715508E236E
:101FD00069D9EF6A000E12008F518F2BEA6A320F17
:101FE000E96E030EEA22FE0EDBCFEFFF1200DECF1A
:101FF00006F0DECF07F0DECF08F0DDCF09F0DD52CE
:10200000DD521200CCEC35F002C0C7F103C0C8F1BC
:1020100004C0C9F105C0CAF11200F86EF4CFF7FF91
:10202000F3CFF6FF040EF626000EF722F822120078
:10203000E552E552F3CF14F0F4CF15F01200FD0E87
:10204000DBCF14F0FE0EDBCF15F01200F36EFE0EA8
:10205000DBCFF4FFF350F45C1200156A8D25146E8B
:102060008E51152214C0E6FF15C0E6FF1200600E67
:10207000EE5C220EEE58C20EEE58010EEE58120023
:10208000CBC1CFF1CCC1D0F1CDC1D1F1CEC1D2F114
:102090001200D950040FE96EDACFEAFF1200D8809F
:1020A000000EEE5412008F51146E156A320E145C3D
:1020B000000E155812000101C651630A12009D88D6
:1020C0009D8A2EDEDF6EDF501200E80EE66E010EF6
:1020D000E66E47EF02F0160EE76FFD0EEA6F420E56
:1020E000E86F120040EC03F0E552E552DF6EDF507E
:1020F0001200FE0EDBCFE6FFE66A1200D3C1E6FF58
:1021000011EF06F0DF50146E050EE15C1200D9509D
:10211000010FE96EDACFEAFF48DE5AEC0CF069EF06
:1021200011F02CDED5EF0EF0E66E3C0EE66E020EE0
:10213000E66E5CEF11F0E76FFD0EE86F060EC2EF82
:102140000EF02EDE41EF0FF02BDEE6521200EDEC2A
:1021500000F0E552E552D4EF01F010DE4FEF10F041
:102160000A0E0B6E0C6A0D6A0E6AEECF06F0EECF09
:1021700007F0EECF08F0EFCF09F01200E76EFD0E8A
:10218000DBCFE9FFFE0EDBCFEAFFE750E926000ECA
:10219000EA221200E66EE66AE66A21EC2AF0E8EF2F
:1021A0000EF0ECDD000EEE5C1200E96EFF0EDA20A0
:1021B000EA6E1200D9CFE6FFDACFE6FF1200DEDDCD
:1021C000800EEE5C1200DADDD8801200D7DDC00E82
:1021D000EE5C0A0EEE58C30EB2EF0FF0FE0EDBCF30
:1021E000E6FF120014C006F015C007F016C008F094
:1021F00017C009F0120097DE43EC09F0E9DD6CEF3F
:102200000FF0FD0EE96F070EC2EF0EF0C9DD050EEF
:10221000E1261200C5DDDEEF0EF0C2DDFE0EDB5062
:102220001200D9CFE9FFDACFEAFF1200B9DD040EC0
:10223000E1261200A3DD400EEE5C12000101010E4A
:10224000D96F1200E66E16DEE5EC34F0146E090E5E
:102250001200800E0B6E960E0C6E980E0D6E0E6AAE
:102260001200E552E552E5521200C4DD34EC2CF0C8
:1022700018EF10F0DDDDCCEC35F078EF0FF0FD0E4F
:10228000DBCF16F0FE0EDBCF17F0120004EC36F0B9
:10229000C5DD02EF10F0E15E1650146E156AFF0EF8
:1022A000161812008DC0E9FF8EC0EAFF1200E80E7A
:1022B0000B6E030E0C6E1200E66A8DEC07F069EFF0
:1022C00011F0E15E145076DFA7EF10F03DDF5BEF19
:0822D00010F07EDDDF6E12004C
:0822D800ABC2E6FFACC2E6FF59
:1022E000D8EC1BF0E552E552AAC2E6FF99EC1BF0D0
:1022F000E552D9C21DFEB00EE66E020EE66EE0ECAF
:102300001BF0E552E552120061EC17F0E6527FEC4B
:102310001EF00F0E95128314DF6E0301FD6BFE6B32
:10232000FE0EE66E030EE66E640EE66E030EE66EBD
:10233000320EE66EFD0EE66E030EE66E960EE66E4D
:10234000030EE66EDFCFE6FF0EEC2EF0146E0A0EE3
:10235000E15E145072EC19F0D2EC29F09396939848
:102360009394270EE66EE66A5C0EE66E6C0EE66EE1
:10237000000EE66EB00EE66E020E95EC17F002014E
:10238000280EAB6F040EAC6FABC2E6FFE66E62ECDC
:102390001BF0E552E552F3CF64F2F4CF65F202018F
:1023A000180EAA6F1E0ED96F120EAF6F0E01010E1E
:1023B0005B6F0201DA6B7F0EE66EE66AACEC15F03D
:1023C000E552E5527F0EE66E010E8AEC17F07F0EA5
:1023D000E66E020E8AEC17F0760EE66E030E8AECBD
:1023E00017F00201DB6BDC6B0301FC6BE55266EF5F
:1023F00017F061EC17F00301010EFE6FFE0EDBCF4C
:1024000064F366EF17F061EC17F00301020EFE6F44
:10241000FD0EDBCF64F3FE0EDBCF65F366EF17F046
:1024200061EC17F00301050EFE6FFE0EDBCF64F3C7
:10243000FA0EDBCF65F3FB0EDBCF66F3FC0EDBCFD2
:1024400067F3FD0EDBCF68F366EF17F061EC17F072
:102450009DEC17F034EC2CF0E552E552F3CF14F07C
:10246000F4CF15F0010EF3240301FE6F310EE66E7A
:10247000E66A9DEC17F0640EE66E030E8FEC17F023
:10248000E15E145066EF17F061EC17F080EC17F086
:1024900042EC2CF0E552E552E55207C014F008C0BA
:1024A00015F009C016F0142A000E1522162214C0C9
:1024B000FEF3310EE66EE66A80EC17F0640EE66E0F
:1024C000030E95EC17F066EF17F0E6687F0EE66EE8
:1024D000E66AE66AE66A2AEC33F0050EE15EF3CFBF
:1024E000DBF2F4CFDCF21200DBC2E6FFDCC2E6FF77
:1024F0008ADFE552E552120061EC17F0080EE12682
:102500000201DE5102E1010EDE6F0301FD5101E126
:102510001CD3030196513C0A01E108D30C0A01E1E6
:102520006FD1010A01E16CD1030A01E169D1010A0D
:1025300001E166D1070A01E163D1010A01E160D13D
:10254000030A01E15DD10E0A01E15AD1010A01E15C
:1025500057D1030A01E154D1010A01E151D10C0A1A
:1025600001E14ED10A0A01E14BD1030A01E148D150
:10257000010A01E145D17F0A01E142D1010A01E1ED
:102580003FD1030A01E13CD1010A01E139D1070A37
:1025900001E136D1010A01E133D1030A01E130D171
:1025A000010A01E12DD10F0A01E12AD1010A01E15D
:1025B00027D1030A01E124D1010A01E121D1070A4F
:1025C00001E11ED1010A01E11BD1030A01E118D189
:1025D000690A01E110D1010A01E108D1020A01E111
:1025E00002D1070A01E1FAD03E0A01E1F4D0010A62
:1025F00001E1EED0390A01E1E8D03E0A01E1D8D08C
:10260000010A01E1CBD00A0A01E1C2D01F0A01E1AF
:10261000BBD0180A01E1B0D0010A01E1A6D0340A0A
:1026200001E1A0D0370A01E19AD0010A01E194D07A
:10263000070A01E18ED0010A01E188D0030A01E115
:1026400082D0300A01E17DD0010A01E178D03E0A52
:102650006DE0010A57E0120A4FE0010A45E0150A51
:1026600040E0120A39E0010A34E0030A24E00E0ACD
:1026700017E0030A01E1ACD0070A0FE0010A0AE003
:102680001A0A05E0190A01E060D226DE5ED252EC99
:102690001CF05BD259EC1CF096D0BAEC1DF055D270
:1026A00026EC1DF0000901E081D0F0EC1DF00009DE
:1026B00001E186D07BD0270EABEC17F0B00EE66EB2
:1026C000020E8FEC17F0E15E14500301010EFC6F57
:1026D0003CD297C3AAF239D297C3ABF298C3ACF2FB
:1026E00034D297C3D9F231D2500EE66E6C0EE66E3C
:1026F000000EE66EC9DE4FD098C3E6FF97C3E6FF33
:102700002BDA4AD097C3E6FF98C3E6FF62EC1BF0D2
:10271000E552E552F3CF16FEF4CF17FE99C31CFE27
:102720000E0111890201010EDA6F0FD20201DA5196
:1027300001E10BD20E0111990201DA6B06D2C5DE5E
:1027400004D2D2DE02D297C36EFFFFD197C36FFFD0
:10275000FCD197C370FFF9D197C371FFF6D197C32E
:1027600072FFF3D197C35BFEF0D1100EABEC17F004
:10277000940EE66E020E06D0040EABEC17F0A50E1A
:10278000E66E020ECCDBDFD166DB7BEC19F003D00A
:1027900062DBD4EC19F0E552E55230D026EC1DF0A6
:1027A000000904E1F0EC1DF000090AE0010E0BD075
:1027B00030EC1DF0000906E1F6EC1DF0000902E125
:1027C000000E01D0010EE66E18D073CFE6FF15D0D3
:1027D00007EC1DF0BAD11FEC1DF0B7D1958E959C7A
:1027E0000301FA81B2D10301FA83AFD197C3FBF39E
:1027F00096908490AAD1FCC3E6FFFBDDE552A5D1FB
:10280000030E97C3DBFF040E98C3DBFF050E99C3CD
:10281000DBFF060E9AC3DBFF010EF36E070EF3CF4C
:10282000DBFF96514E0A01E161D1030A01E15BD160
:10283000010A01E155D1070A01E14FD1010A01E185
:102840003ED1030A01E133D1010A01E112D10F0A9D
:1028500001E105D1010A01E1FFD0030A01E1F9D04C
:10286000010A01E1ECD0070A01E1D1D0010A01E13E
:10287000C4D0030A01E1BDD0010A01E1B1D07F0A51
:1028800001E1A5D0010A01E195D0030A01E185D05B
:102890000A0A01E17FD00C0A01E179D0010A01E1C5
:1028A00073D0030A62E0010A59E00E0A51E0030AFC
:1028B00048E0010A42E0070A31E0010A28E0030A81
:1028C0001FE0010A01E018D160DB01E215D1030E1F
:1028D000DBCFDDF2DDC2E6FF0FEC07F0E552E76E7D
:1028E000070EE7CFDBFFDB5002E00201DD6BDDC24C
:1028F000E6FF050EE66E93EC1EF0E552E552FCD0C5
:1029000044DB01E2F9D047DB37EC07F0DED02ADB0D
:1029100001E3F2D0C1DA5FEC07F0D6D096DA800E90
:10292000EE5C960EEE58980EEE58000EEE5801E34F
:10293000E3D02EDB8DEC07F00ED02ADB5AEC0CF046
:102940000AD010DB01E3D8D0A7DABCEC07F0BCD08A
:102950001FDB30EC0DF0E552E552B6D016DB01E29C
:10296000CBD019DB34EC0DF0B0D06FDA000EEE5C9A
:10297000000EEE58010EEE58000EEE5801E3BCD0EA
:102980008BDA64EC0DF0A0D08FEC0DF0B1D0A4EC9C
:102990000DF0AED0B9EC0DF0ABD0030EDBCF83F071
:1029A000040EDBCF84F0050EDBCF85F0060EDBCF07
:1029B00086F043D0030EDBCF87F0040EDBCF88F028
:1029C000050EDBCF89F0060EDBCF8AF036D083C050
:1029D000DAF184C0DBF185C0DCF186C0DDF113D013
:1029E00087C0DAF188C0DBF189C0DCF18AC0DDF193
:1029F0000AD0030EDBCF82F020D082C0DAF10101D1
:102A0000DB6BDC6BDD6B0101020ED96F4DD0030E69
:102A1000DBCF14F0040EDBCF15F0050EDBCF16F084
:102A2000060EDBCF17F0145015101610171002E128
:102A3000000E01D0010E00018C6F010E49D005DAA5
:102A4000210EEE5C000E2DDA38E2A5DAD4EC0DF0A2
:102A50003CD0EDEC0DF04CD006EC0EF049D0F5D9A1
:102A6000000EEE5C010E1DDA28E295DA1FEC0EF086
:102A70002CD0010E69DA04E00001010EE56F02D0EE
:102A80000001E56B020E60DA04E00001010EE66F62
:102A900002D00001E66B040E57DA04E00001010EDB
:102AA000E76F02D00001E76B070EDB6A25D060DA22
:102AB00004E2F2D938EC0EF007D0030E09D058DA50
:102AC00006E2EAD95FEC0EF0E552E55211D0030EB2
:102AD000F36E070EF3CFDBFF0FD079EC0EF008D0CA
:102AE00090EC0EF005D0A7EC0EF002D0C8EC0DF083
:102AF000E76E070EE7CFDBFF070EDB5004E0070EA3
:102B0000DBCFDEF209D00101D95103E0D9C1DEF2F9
:102B100003D00201010EDE6F0201DE0516E10001A5
:102B20008B5113E00201020EDE6F0FD0DAC1E6FF17
:102B3000DBC1E6FFDCC1E6FFDDC1E6FFDEC2E6FF8A
:102B40006FDC146E050EE15E1450080EE15C02E2CB
:102B5000E16AE552E16EBAD1B4D9020EE126819460
:102B60008198FE0EDB50020B020802E0000E01D03D
:102B7000010EE8B08186E8A0819681888198FE0EDA
:102B8000DB50010BE8B08186E8A0819681888198AE
:102B9000DE52800EDD6E080EDF6EDF501EE0010E8D
:102BA000DBCFE6FFFD0EDB50E552E714146E010E9D
:102BB000DB50145C02E0000E01D0010EE8B081860B
:102BC000E8A0819681888198010EDBCFF3FFF39016
:102BD000F342F3CFDBFFDF06E0D78184020EE15C36
:102BE00002E2E16AE552E16E71D10301FAA113D16B
:102BF000030E0101C65D01E094D00301FF51030AF9
:102C00006CE0010A50E0030A2AE0010A06E0FF6BCB
:102C1000020EFA1501E182D07ED0020EFA1504E010
:102C20006BD906E0010E04D08350800B01E0010E49
:102C300000090EE0010EFF6F0E01140E5C6FCFC194
:102C4000E6FFD0C1E6FFD1C1E6FFD2C1E6FF96D1D3
:102C5000020EFA1502E0838C010C839C000C020E1C
:102C6000FA1504E049D906E0010E04D08350800B28
:102C700001E0010E00090AE1FF6B020EFA1503E004
:102C8000838C010E02D0839C000E24D10E015C5176
:102C900001E0DAD00301020EFF6FFA1502E0839C17
:102CA000000C838C010C020EFA1504E025D906E015
:102CB000010E04D08350800B01E0010E000901E0F9
:102CC000C3D0030EFF6F020EFA1502E0838C01D011
:102CD000839C0E01010E5C6F1200020EFA1504E0D7
:102CE0000BD906E0010E04D08350800B01E0010EE9
:102CF000000908E0020EFF6FFA1502E0839C000C49
:102D0000838C010C0E015C5101E09ED00301FF6B2E
:102D1000020EFA1503E0838C010E02D0839C000E94
:102D2000D9D00301FB5160E0FF51030A3AE0010AE8
:102D300025E0020A05E0FF6B020EFA1565E052D0AD
:102D4000020EFA1504E0D8D806E0010E04D0835034
:102D5000800B01E0010E000909E0020EFF6F849074
:102D6000FA1502E0839C000C838C010C020EFA150C
:102D700002E0838C01D0839C84901200020EFA152D
:102D800004E0BAD806E0010E04D08350800B01E0C5
:102D9000010E000959E1030EFF6F8480FBC35CFE46
:102DA0001200020EFA1504E0A7D806E0010E04D0C6
:102DB0008350800B01E0010E000907E0020EFF6F57
:102DC0008490FA150BE0839C000C0E015C513CE1F1
:102DD0000301FF6B8490020EFA1502E0838C010C54
:102DE000839C000C838C010C020EFA1504E084D83D
:102DF00006E0010E04D08350800B01E0010E0009B3
:102E000005E0020EFA1505E0839C000C020EFA158F
:102E100012E0838C010C020EFA1504E06DD806E076
:102E2000010E04D08350800B01E0010E000905E083
:102E3000020EFA1505E0839C000C020EFA1502E062
:102E4000838C010C839C000E1200D950030FE96E95
:102E5000DACFEAFF1200030E7ED8D9CFE6FFDACF31
:102E6000E6FF83EC2BF0146E060EE15E1450020EAA
:102E7000DBCFE6FFDECFE6FFDDCFE6FF1200EE5050
:102E80001416EE501516EE501616EE501716145076
:102E900015101610171012007ED8040EDBCFE6FFB7
:102EA0001200EE58000EEE58000EEE581200D880B8
:102EB000FF0EEE54000EEE54000EEE54000EEE54D3
:102EC0001200D9CFE6FFE1CFD9FF1200E552E7CFDC
:102ED000D9FF1200CBC1E6FFCCC1E6FFCDC1E6FFB2
:102EE000CEC1E6FF4BD0EECFE6FFEECFE6FFEECF52
:102EF000E6FFEFCFE6FF12008350800B800A12003E
:102F0000FC0EDBCFE6FFFD0EDBCFE6FFFE0EDBCFD8
:102F1000E6FF1200E66E20DEE552E5521200E66E94
:102F200067EC2CF0146E060E1200E66E95EC2CF099
:102F3000146E070EE15E14501200FD0EDBCFE6FFAB
:102F4000FE0EDBCFE6FF1200146E156A166A176AD2
:102F50007CDF3FEF17F0E66EE66A970EE66E030E33
:102F6000E66E120072DF100EEE5C270E51EF17F0C6
:102F70006CDFFF0EEE5CFF0E51EF17F0B1EC04F0CA
:102F8000E552E552E552E55212005FDF57EF17F0C8
:0E2F90005CDF73EF17F0030EDBCFE6FF1200DD
:022F9E00F36AD4
:102FA000F46AFF0EE124E96EFF0EE220EA6EED66A0
:102FB00007D02F0EEF6404D03A0EEF6001D0F32A51
:102FC0001200F36AF46AFF0EE124E96EFF0EE220BC
:102FD000EA6EED660AD0200EEF5C06E0080EEF64A4
:0C2FE00004D00E0EEF6001D0F32A1200A6
:042FEC00303132331B
:0D2FF0003435363738396162636465660038
:022FFE001200BF
:1030000000000000000000000000000000000000C0
:1030100000000000000000000000000000000000B0
:1030200000000000000000000000000000000000A0
:103030000000000000000000000000000000000090
:103040000000000000000000000000000000000080
:103050000000000000000000000000000000000070
:103060000000000000000000000000000000000060
:103070000000000000000000000000000000000050
:103080000000000000000000000000000000000040
:103090000000000000000000000000000000000030
:1030A0000000000000000000000000000000000020
:1030B0000000000000000000000000000000000010
:1030C0000000000000000000000000000000000000
:1030D00000000000000000000000000000000000F0
:1030E00000000000000000000000000000000000E0
:1030F00000000000000000000000000000000000D0
:1031000000000000000000000000000000000000BF
:1031100000000000000000000000000000000000AF
:10312000000000000000000000000000000000009F
:10313000000000000000000000000000000000008F
:10314000000000000000000000000000000000007F
:10315000000000000000000000000000000000006F
:10316000000000000000000000000000000000005F
:10317000000000000000000000000000000000004F
:10318000D0EC20F01468156AFD0EDBCF08F0FE0EBF
:10319000DBCF09F014C00DF015C00EF05FEC36F077
:1031A00008C0DEFF09C0DDFF48EC20F009E0E66A58
:1031B00048EC36F0E552DF06010EF6E2DB06F4D706
:1031C000D8EC1FF00D680E6A14C008F015C009F0A5
:1031D0005FEC36F004C014F005C015F004C0DEFF4B
:1031E00005C0DDFF48EC20F005E0DFCFE6FF48EC4E
:1031F00036F0E552020EE15C02E2E16AE552E16E70
:10320000D5EF1EF0010ED16E1200D16A120002013C
:10321000635101E1040012000201010E636F12000C
:10322000A5EC20F04EEC1FF0FB0EDBCFEEFFFC0E0A
:10323000DBCFEDFFDF5001E09D80E552D5EF1EF0C2
:10324000D0EC1EF0030EAFEC20F0EDCFDBFFDF5033
:1032500001E09D804FEC20F014C0F3FF15C0F4FF97
:10326000030EE15C02E2E16AE552E16ED5EF1EF089
:10327000A5EC20F04EEC1FF0F90EDBCFEEFFFA0EBE
:10328000DBCFEEFFFB0EDBCFEEFFFC0EDBCFEEFF66
:10329000DF5001E09D80E552D5EF1EF0D0EC1EF02E
:1032A000050EAFEC20F0EECFDBFF030EEECFDBFF21
:1032B000040EEECFDBFFDF5001E09D804FEC20F0ED
:1032C000030EDBCF16F0040EDBCF17F014C006F0B0
:1032D00011EC20F0050EE15C02E2E16AE552E16EDC
:1032E000D5EF1EF00201936B93C292F293C27CF26F
:1032F00093C27BF21200A5EC20F002017B29DF6E65
:10330000070EDF5C01E3DF6A7C51DF5C02E1010E46
:103310002ED07B5169EC1FF056EC20F07B5169EC0C
:103320001FF03AEC20F0DFCF7BF2D8EC1FF0000E5C
:103330001416F00E1516145002E1200E15180FE0A9
:10334000FD0EDBCF16F0FE0EDBCF17F0000E1616CB
:10335000F00E171616500AE1100E171807E1FD0EB1
:10336000DB50010B03E10F01010E736F000EE552FC
:10337000D5EF1EF0D0EC1EF002017C517B5D02E126
:10338000010E10D07C5169EC1FF0C9EC1FF07C518C
:1033900069EC1FF0BBEC1FF07C2B070E7C5D01E39A
:1033A0007C6B000ED5EF1EF0A5EC20F002019229F7
:1033B000DF6E070EDF5C01E3DF6A9351DF5C02E141
:1033C000010E0DD0925173EC1FF056EC20F092518B
:1033D00073EC1FF03AEC20F0DFCF92F2000EE552D2
:1033E000D5EF1EF0D0EC1EF002019351925D02E188
:1033F000010E10D0935173EC1FF0C9EC1FF09351E4
:1034000073EC1FF0BBEC1FF0932B070E935D01E3F1
:10341000936B000ED5EF1EF0D0EC1EF0050EE126EA
:1034200015DB000970E1FBEC1FF0A4DF9DEC20F040
:10343000000969E12BEC20F006E2F2EC1EF095DACF
:103440009DEC20F060D0010EDB50C00B2BE054EC63
:103450001FF0DBCF01F2040EDBCF02F2010EDB50D6
:10346000800B0DE036EC1FF0F5CF00F20201046B8B
:10347000056B72CF03F2076B086B066B07D0020176
:10348000C80E006F010E046F056B036B020EDBCFDD
:103490001AFEDBCF57FE2BEC1FF09D900E013689F4
:1034A0009D8031D024EC20F015E1100E151812E1AA
:1034B000020EDBCFE6FF71CFE6FF70CFE6FFB6EC82
:1034C00020F0D890E936EA36E806FBE1A1EC1FF0DF
:1034D0001AE117D024EC20F016E1200E151813E1A4
:1034E000020EDBCFE6FF6FCFE6FF6ECFE6FFB6EC56
:1034F00020F0D890E936EA36E806FBE1A1EC1FF0AF
:1035000002E10F01736B050EE15C02E2E16AE55234
:10351000E16ED5EF1EF0D0EC1EF0050EE126A0DA2C
:10352000000932E1FBEC1FF05DDF9DEC20F00009AB
:103530002BE12BEC20F006E2F2EC1EF047DA9DECDA
:1035400020F022D0010EDB50800B1EE054EC1FF067
:10355000DBCF01F1040EDBCF02F136EC1FF0F5CF2B
:1035600000F10101046B056B72CF03F1076B086B6F
:10357000066B020EDBCF1CFEDBCF59FE2BEC1FF0DF
:103580009D900E01368D9D80050EE15C02E2E16AA0
:10359000E552E16ED5EF1EF0D0EC1EF0FE0EDB50D2
:1035A000200A01E17FD0290A01E17CD0530A70E0B2
:1035B0000E0A64E0770A5AE0670A50E0070A4BE017
:1035C000010A46E0030A41E06B0A37E01A0A2DE0DF
:1035D000090A28E0010A23E00F0A1EE0010A19E0A7
:1035E000030A14E0010A0FE0070A0AE0010A05E0F5
:1035F000030A60E1A2EC20F022D0A2EC20F017D068
:10360000A2EC20F035D088EC20F019D088EC20F026
:103610000ED088EC20F02CD08DEC20F010D08DEC6A
:1036200020F005D08DEC20F023D092EC20F04BEC74
:103630001FF0060EEE6E230E43D092EC20F04BEC02
:103640001FF0B10EEE6E1F0E3BD0A2EC20F008D0A2
:1036500088EC20F005D08DEC20F002D092EC20F028
:103660004BEC1FF0CF0EEE6E2A0E2AD092EC20F01B
:103670004BEC1FF0B80EEE6E260E22D08ADB2D0E1C
:10368000EE6E090E4BEC1FF0890EEE6E0B0E18D08D
:1036900080DB950EEE6E0C0E4BEC1FF0410EEE6EC5
:1036A000100E0ED076DBEE6AED6AC3EC20F0EE6A07
:1036B000ED6A07D0A2EC20F0EEDB450EEE6E120EA6
:1036C000ED6E73D36DDBD8EC1FF0166A176AFD0E32
:1036D0000B6EB50E0C6E060E0D6E0E6A14C006F063
:1036E00011EC20F0CCEC35F002C014F003C015F062
:1036F00004C016F005C017F0800E1526000E162225
:1037000017220B6A0C6A010E0D6E0E6A02C006F0DB
:1037100011EC20F0D8EC31F006C014F007C015F021
:1037200008C016F009C017F006C0F3FF07C0F4FF89
:103730003CD3A5EC20F0050EF36EFE0EDBCFF4FFBC
:10374000F350F45C05E2050EF36EFE0EF3CFDBFFE3
:10375000FE0EDB50166E176AFE0EDB5031EC20F0C9
:1037600014C008F015C009F016C00DF017C00EF017
:103770005FEC36F00850DF6EDFCF37FE0E013751B9
:10378000E8240E01386F030E0E013703F3CF39FE24
:10379000040E3703F3CF3AFEDF5031EC20F014C0B3
:1037A00009F0DFCF0EF093EC36F00950E552FDD270
:1037B000F7DA97EC20F0F3CF64F2F4CF65F2F5D2AC
:1037C000EFDA040EE1269D900E0136919D800E01E8
:1037D000C80E446F030E456F020E44CEDBFF030E8E
:1037E00045CEDBFFDF6ADF6ADF509BDBEF503BE05B
:1037F000310EDF5C38E2DF5094DBEF507F0BE76E79
:10380000010EE7CFDBFFDBCF14F05F0EE76E14187D
:10381000E8AE02D0143403D0E750D88014540AE242
:10382000200E146E010EDBCFE7FF1450E75E010E91
:10383000E7CFDBFF040E146E4E0E156E000E166EF3
:10384000010EDBCF17F0186A196A17AE02D018689C
:10385000196872EC20F0F550E66EB1DBE552E750E6
:10386000EF6EDF2AC1D7ABDBEF6A0E01466B64C295
:1038700018FE65C219FE9D903F0E0E0111170E0134
:1038800036819D80040EE15C02E2E16AE552E16E60
:103890008CD2A8EC20F089D2A8EC20F00E0136B131
:1038A000FDD783D29D900E0136910E01119D9D8012
:1038B0001200400E0E011115146E010E0E01361588
:1038C00014101200A5EC20F0DF6A68EC20F008006C
:1038D000F55010E0F90EDB50DF5C0CE26ADAD950EB
:1038E000FD0FCEDBEF22D950FA0FCADBEE22EE221B
:1038F000DF2AEBD75EDAE55258D252DAFE0EDB5001
:10390000040A32E0070A1CE0010A0EE0030A2CE177
:103910009D900E0136990E011191EFDA000EE66EC0
:10392000020E58DB98DA20D09D900E01369B0E01D6
:103930001195E3DA630EE66E010E4CDBF7DA14D074
:103940009D900E01369D0E011199D7DA000EE66E9C
:10395000010E40DB0E01000E4B6F010E4C6F0E018D
:10396000000E536F010E546F20D2EFDBDF6A4FD889
:1039700068DA5EDB09E065DAF4DA010E14DBDBCF2E
:103980001AFEDBCF57FEDF88BCDB52DB18E0B9DB69
:103990000900F5500900F5CFE7FF0800F5CFF8FF63
:1039A000E7CFF7FFF66E0800F55009E0AADBD9DA99
:1039B000020EF9DADBCF1BFEDBCF58FEDF8A9D90CB
:1039C000DF500E0136139D80E552EFD1E9D937D88B
:1039D00038DA2EDB0CE035DAC4DA030EE4DADBCFBA
:1039E0001CFEDBCF59FE9D900E01368D9D80DDD1F2
:1039F000D7D90DD89CDBF3CF12FEF4CF13FEFC0E0B
:103A0000DBCF1AFE9D900E0111819D80CED19D903D
:103A1000CF0E0E013617FA0E0E0111179D801200FF
:103A2000BFD90DD884DBF3CF16FEF4CF17FEFC0E02
:103A3000DBCF1CFE9D900E0111899D80B6D19D901B
:103A40000E01369D0E0111999D801200300E0E015F
:103A5000361505E1050E0E01111501E1000C010CF2
:103A6000400E0E01361505E1100E0E01111501E193
:103A7000000C010C6ADBCBDF4DDA34EC2CF0E552A4
:103A8000E552110EF35C000EF45803E3100E49DA10
:103A9000EF6A0E01000E476F020E486F0E01630EB3
:103AA000496F010E4A6FFD0EDBCFE9FFDB2AFE0EE8
:103AB000DBCFEAFF01E3DB2AEFCFDFFFDF5028E0B7
:103AC00090DAFC0E67DB92DAEE52E9CF14F0EACF1F
:103AD00015F0E9CFE6FFEACFE6FF83DAEE52E9CF51
:103AE00016F0EACF17F0E9CFE6FFEACFE6FFDFCF27
:103AF000E6FF52DD186E050EE15E185087DA71DAC6
:103B0000FB0E48DB3ADBEE52EE6AED6A7FDACBD78A
:103B100068DAEF6A32DBEF6A69DAEE52EE6AED6A72
:103B20009AD904DAFA0EDBCF1BFE1BCE1AFEDBCFCE
:103B300058FE58CE57FE9D90300E0E0136139D80D4
:103B4000E55233D12DD963DF140EE66E0E0EE66E0C
:103B5000120EE66E0E0EE66EFE0EDBCFE6FF1CDDED
:103B6000146E050EE15E14509D90050E0E011113AA
:103B70009D801BD14CDF0201640E006F0101636F59
:103B80000201950E016F0C0E026F0101410E646F70
:103B9000100E656F0201640E036F0101666F020172
:103BA000046B056B0101676B686B0201066B010119
:103BB000696B010E0201076F086B01016A6F6B6B85
:103BC0004AD9B4D99D90300E0E0136139D80120053
:103BD000300E0E0136151200400E0E013615120081
:103BE00002017C517B5D01E1000C010C020193514B
:103BF000925D01E1000C010CA8DAFE0EDBCFE6FFBE
:103C0000E66ACFEC17F0E552E552F350F41004E009
:103C1000FE0EDB50D00F04D0FE0EDB50BF0F0A0F9C
:103C2000DF6EDF50E552C1D0BBDAFD0EDBCFDEFF29
:103C3000DBCFDDFF04DAEF5005E0DF2A010EFAE307
:103C4000DB2AF8D7FCD9FC0EDBCFEFFFF8D9010E49
:103C5000B0DAEF6AADD914C0F3FF15C0F4FF020E5D
:103C6000E15C02E2E16AE552E16E9FD09D929F82A3
:103C7000D08EF90E94160F0EBD6EBA6E1C0ECA6E63
:103C8000CB680E01116B0E017F0E1E6F0E011A6FB5
:103C90000E011B6F0E011C6F0E011D6F0E01370E02
:103CA000126F1A0E136F0E01370E146F1A0E156F66
:103CB0000E01370E166F1A0E176F0E01370E186FA2
:103CC0001A0E196F1200810ECD6E9F90140EE66EC3
:103CD00030DDE552E80EE66E030EE66E69DDE55274
:103CE000E5520E017F0E5A6F5ACE59FE5ACE58FE3B
:103CF0005ACE57FE0E01366B0E013B6B1200870E3B
:103D0000D56EB16AF18EF26A9D6AA06AAFDF63EF89
:103D10001EF046D8AA6AFE0EDB50A96EA69EA69C8F
:103D2000A680A85042D03CDAA198AA6AFE0EDB50C9
:103D3000A96EFD0EDB50A86EA69EA69CA684F2502E
:103D4000800B01E0010EDF6EF250400B01E0010E2E
:103D5000E76E010EE7CFDBFFF29EF29C550EA76ED9
:103D6000AA0EA76EA682DF50E8B0F28EE8A0F29EFF
:103D7000010EDB50E8B0F28CE8A0F29CA1A8FED7BF
:103D8000A198A694020EE15C02E2E16AE552E16EBE
:103D90000CD0FC0EDBCFE9FFFD0EDBCFEAFF1200FB
:103DA000D9CFE6FFE1CFD9FF1200E552E7CFD9FF27
:103DB00012008ED90800F550E66E83D9E552E7501F
:103DC000EF6E86D90900F5CF14F00900F5CF15F094
:103DD0000800F5CF16F075D9EE5215C0EEFF16C0EB
:103DE000EDFF1200020EDBCFE6FF390E176E520E0A
:103DF000186E000E196EDECF1AF0DDCF1BF01C6AB4
:103E0000060E0C6E0D6A0E6A1AC007F01BC008F091
:103E10001CC009F00CEC32F004C01AF005C01BF015
:103E200006C01CF017500424146E18500520156E9F
:103E300019500620166E14C0E6FF15C0E6FFE66EA8
:103E40001200FC0EDBCFF6FFFD0EDBCFF7FFFE0E00
:103E5000DBCFF8FF12000E01000E476F020E486F15
:103E60000E01000E4F6F020E506F12009B0E146E6B
:103E7000530E156E000E166EDECF17F0DDCF18F064
:103E80001838186A0F0B176E070E1716000E181643
:103E9000196A72EF20F0ED6EC3EF20F09D50010B18
:103EA000DF6E9D9061EF20F07FD9FF0E14160F0E8C
:103EB000151614C0E6FF15C0E6FF62EC1BF0E552D4
:103EC000E552030EF3CFDBFF040EF4CFDBFF030E4E
:103ED0001200030DF3CFE9FFF4CFEAFF660EE926E7
:103EE000020EEA221200030DF3CFE9FFF4CFEAFF3E
:103EF0007D0EE926020EEA2212009D80210EE66E5A
:103F0000FB0EDBCFE6FFFC0EDBCFE6FFFD0EDBCFCB
:103F1000E6FF1200FD0EDBCFE6FFFE0EDBCFE6FF75
:103F20001200E76ECED8E750D9EF20F00E01630EF5
:103F3000496F010E4A6F0E01630E516F010E526FF1
:103F40001200740EE9260F0EEA22EECFE6FFEFCF45
:103F5000E6FF90DD146E050EE15E1450DF50010B9C
:103F600012000900F5CFE6FF0900F5CFE6FF0800D3
:103F7000F5CFE6FF1200020E1CD9EF50E66EFB0EE5
:103F8000DBCFE9FFFC0EDBCFEAFFE552E750EF6E37
:103F90001200EECF14F0EECF15F093D814C0EEFF60
:103FA00015C0EDFF1200E66EA8DCC7D8FB0E1200AC
:103FB000FD0EDBCF14F0FE0EDBCF15F01200DF504C
:103FC000E76E020EDBCFE9FF030EDBCFEAFFE7501F
:103FD000D9EF20F0E66E76DC146E060EE15E14502A
:103FE000120047CEE9FF48CEEAFF120049CEE9FFB2
:103FF0004ACEEAFF1200D950020FE66E000EDA2018
:10400000E66ED9CFE6FFDACFE6FF12000E01030E0F
:104010004727000E48230E01030E4927000E4A23AE
:10402000120015C007F016C008F017C009F0120002
:104030000900F5500900F5100800F5101200DECF58
:10404000E9FFDDCFEAFF1200AFD8000E1416F00E24
:10405000151614501200A8D83B0E145C000E15580B
:104060001200156AE8307F0B146EF00E1426000E55
:1040700015221200020E9DD8FC0EDBCFEFFF1200BE
:10408000E96EFF0EDA20EA6E030EEE26000E120035
:10409000D9CFE9FFDACFEAFFEE50ED101200010EA2
:1040A000DBCF14F0020EDBCF15F01200FD0EDBCFDC
:1040B000EEFFFE0EDBCFEDFF1200450EEE6E120E90
:1040C0001200FD0EDBCFE9FFFE0EDBCFEAFF120090
:1040D000FA0EDBCFF6FFFB0EDBCFF7FFFC0EDBCFDC
:1040E000F8FF120014501724F36E15501820F46EC8
:1040F00016501920F86EF4CFF7FFF3CFF6FF080043
:1041000012009FDE030EF626000EF722F8221200A0
:1041100040DE2F0EEE6E140E12003BDE560EEE6EDB
:10412000160E120036DEAB0EEE6E180E1200F2DE28
:1041300062EC1BF0E552E5521200E552E552E55201
:10414000E552120026DE5DEF20F02ADEE652120074
:1041500027DEE0DEE0EC1BF0E552E5521200E1263E
:104160009DDE010EEECFDBFF020E120068DF010EB6
:10417000E916000EEA16010E120033DFEE52EE6A67
:10418000ED6AF6EF1FF0FA0EDBCFE9FFFB0EDBCF97
:10419000EAFF1200DBCFEFFF29DFDBCFEFFF1200DA
:1041A000FFDD020EE1261200DECF14F0DDCF15F0A8
:0A41B0001200E926000EEA221200B8
:0641BA0019EC26F0FB0EDB
:1041C000DBCFF3FFDB06F35000090AE067EC26F0D3
:1041D000FA0ED2EC26F0F3E1151CF1E1010E01D04C
:1041E000000E48EF26F019EC26F03B0EE12402E326
:1041F000E168E652E16E010EDB6A020EDB6AF90E3F
:10420000DBCFF6FFFA0EDBCFF7FFFB0EDBCFF8FFBD
:104210000800F550DF6EDF5002E16CEF25F0250E4F
:10422000DF5C02E05FEF25F0030EDB6A040EDB6A61
:10423000050EDB6A060EDB6A070EDB6A81EC25F0F1
:104240002D0EDF5C0CE02B0EDF5C09E0200EDF5C46
:1042500006E0230EDF5C03E0300EDF5C1AE1DF5086
:10426000300A14E0130A0FE0030A0AE00B0A05E023
:10427000060AE4E1030EDB80E1D7030EDB82DED722
:10428000030EDB84DBD7030EDB86D8D7030EDB8877
:10429000D5D72A0EDF5C1BE17DEC25F0CBEC25F0B9
:1042A00010E0030EDB8008680968130EDBCF0DF009
:1042B000140EDBCF0EF055EC32F0040E06C0DBFF1F
:1042C00003D0130EB4EC25F081EC25F00BD0090ED1
:1042D000DB6A22EC26F003E096EC26F0FAD7090E12
:1042E000B4EC25F0030EDBB0DB982E0EDF5C1BE197
:1042F00081EC25F02A0EDF5C0BE17DEC25F0CBECA8
:1043000025F003E1130E06EC26F081EC25F00BD02E
:10431000090EDB6A22EC26F003E096EC26F0FAD7D1
:10432000090E06EC26F0680EDF5C07E181EC25F053
:10433000680EDF5C1DE1030E18D0740EDF5C17E021
:104340007A0EDF5C14E0480EDF5C06E0540EDF5CA2
:1043500003E05A0EDF5C02E1020E07D06C0EDF5C58
:1043600003E06A0EDF5C04E1010E59EC26F0C9DBC4
:10437000DF506E0A01E17FD31E0A01E192D1200ACB
:1043800001E18FD13F0A01E149D11A0A01E146D189
:104390000D0A01E143D1200A01E140D13A0A01E1CD
:1043A0003DD1200A01E13AD1260A01E135D10D0AB9
:1043B00001E132D11A0A01E1D9D0200A4AE0300ADB
:1043C0001FE0460A0EE0250A01E083D3D950F90F19
:1043D000E96EFF0EDA20EA6E010EEE5E000EEE5A76
:1043E000EE5A67EC26F0250EE66E95DB03E1151C10
:1043F00001E169D363EC26F001E26BD3DB2A69D3D8
:10440000080EDB6A040EDB50010806E2040EDB0432
:104410002BEC26F0DB508BDB080EDB5009E0030EA3
:10442000DB50010B05E172DB01E04DD3080EDB6AC6
:1044300064DBEFCFDFFFDBEC26F003E1151C01E1CD
:1044400042D363EC26F001E3DB2A60DB01E141D3D8
:104450003AD3070EDB5002080FE1A7EC26F0030E5B
:104460006EEC26F00E0EEECFDBFF0F0EEECFDBFF75
:10447000100EEECFDBFF20D0F70EDBCF17F0F80EDB
:10448000DBCF18F0020E175E000E185AF70E17C099
:10449000DBFFF80E18C0DBFF17C0E9FF18C0EAFF0A
:1044A0005EEC26F0166A0E0E14C0DBFF0F0E15C070
:1044B000DBFF100E16C0DBFF0E0EDBCFE6FF0F0E8C
:1044C000DBCFE6FF100EDBCFE6FF42EC2CF0E5522F
:1044D000E552E552130E07C0DBFF140E08C0DBFFE8
:1044E000060EDB5005E0130EA2EC26F001E26ADBBB
:1044F000C6EC26F002E2130E37DB89EC26F006E06C
:10450000040EA2EC26F002E2050E2EDB030EDBB059
:1045100005D0FCDA01E0D7D2080EDB6A090EDB6AAF
:104520000E0EDBCFF6FF0F0EDBCFF7FF100EDBCF4B
:10453000F8FF0800F550DF6EDF5014E0CCEC26F0F9
:1045400011E2DBEC26F003E1151C01E1BCD2BBDB80
:1045500001E3DB2A090EDB2AD9500E0FE96E000EAB
:10456000CBDBE7D7D3DA01E1B4D2ADD2C6DA110E94
:10457000EECFDBFF120EEDCFDBFF110EDBCFE6FF40
:10458000120EDBCFE6FF34EC2CF0E552E552130EB1
:10459000F3CFDBFF140EF4CFDBFF060EDB5004E09D
:1045A000130ED0DB01E20EDBC6EC26F002E2130EA6
:1045B000DBDAAFDB05E0040EC5DB02E2050ED4DA80
:1045C000030EDBB005D0A2DA01E07DD2080EDB6A73
:1045D000090EDB6A110EDBCFE9FF120EDBCFEAFF1B
:1045E000EFCFDFFFDF5014E0D7DB12E2E4DB03E1C3
:1045F000151C01E168D267DB01E3DB2A090EDB2A27
:10460000110EDB2ADBCFE9FF120EE8E3DB2AE6D747
:104610007DDA01E15ED257D2030EDB8E070EDB049A
:1046200010E195DB040E5ADB0A0EEECFDBFF0B0E1A
:10463000EECFDBFF0C0EEECFDBFF0D0EEECFDBFF80
:104640006CD0070EDB5003082CE1030EDBAE0DD05F
:10465000B2DA020E76DAEFCF14F0156A166A176A2C
:1046600014AE39D01568166835D0F70EDBCF15F0CB
:10467000F80EDBCF16F0020E155E000E165AF70E7E
:1046800015C0DBFFF80E16C0DBFF15C0E9FF16C032
:10469000EAFFEFCF14F00A0E14C0DBFF0B0EDB6A4B
:1046A00038D0070EDB50020809E1030EDBAE04D060
:1046B00059DB16AE10D00ED055DB0DD0030EDBAE9D
:1046C00012D079DA020E3DDAF9DA166A176A15AEF7
:1046D00002D016681768E2DA0C0E16C0DBFF0D0E6A
:1046E00017C0DBFF1AD0F70EDBCF16F0F80EDBCFCA
:1046F00017F0020E165E000E175AF70E16C0DBFFFB
:10470000F80E17C0DBFF16C0E9FF17C0EAFFD6DAC4
:10471000C5DA0C0EDB6A0D0EDB6A060EDB5005E116
:10472000010EF36E050EF3CFDBFF150EDB6A160EDE
:10473000DB6AD950370F146E000EDA20156E390E71
:1047400014C0DBFF3A0E15C0DBFF380EDB6A080E23
:10475000DB6A0A0EAEDADF50780A12E0200A10E0B7
:10476000280A0CE0200A0AE03F0A06E00D0A02E0EF
:10477000200A08E1020E05D0080E03D0080EDF263D
:10478000100E97DA030EDBBE02D0DB92DB94DB5017
:10479000800B24E08ADAD890030EEB50000A08E67A
:1047A000000EEE5C000EEE58000EEE58000EEE58B5
:1047B00015E213DA0B680C680D680E68CCEC35F066
:1047C0000A0E02C0DBFF0B0E03C0DBFF0C0E04C0A1
:1047D000DBFF0D0E05C0DBFF2D0E08D0030EDBA2A4
:1047E00002D02B0E03D0DBA408D0200EF36E170EE0
:1047F000F3CFDBFF150EDB2A02D0170EDB6A050EA6
:10480000DB5003E1B7D901E189D0EC0E146E2F0E15
:10481000156E000E166E070EDBCF17F0186A196AB8
:104820001A6A17C00BF018C00CF019C00DF01AC0AE
:104830000EF0D3D904EC36F014500224F36E155068
:104840000320F46E16500420F86EF4CFF7FFF3CF78
:10485000F6FF0800090EF5CFDBFF580EDF5C0FE115
:10486000610EF36E090E7BD90AE3200E146E090E59
:10487000DBCFE7FF1450E75E090EE7CFDBFF070E43
:10488000DBCF14F0156A166A176A0FDA14C00BF042
:1048900015C00CF016C00DF017C00EF0EECF06F0EC
:1048A000EECF07F0EECF08F0EFCF09F004EC36F0D2
:1048B00009C0EDFF08C0EDFF07C0EDFF06C0EFFF28
:1048C000390EDBCFE9FFDB063A0EDBCFEAFF01E270
:1048D000DB06090EDBCFEFFF150EDB2A4BD995E186
:1048E000030EDBA61DD06F0EDF5C06E1C1D918E315
:1048F000150EDB285BDA14D0780EDF5C09E0580E69
:10490000DF5C06E0620EDF5C03E0420EDF5C08E184
:10491000020EF36E160EF3CFDBFF02D0150EDB6A2C
:10492000030EDB50100B0EE0040EDBCF14F0050E6F
:10493000DB50D880145406E2060EDB5003E1040E6F
:10494000DB5034DA95D90AE2050EDBCFE7FF150E0E
:10495000DB50E75E050EE7CFDBFF02D0050EDB6A1A
:10496000040EDBCF14F0160E45D9D880145414E28F
:10497000160EDBCFE6FF150EDBCFE6FF040EDBCF16
:10498000E6FF050EDB50E552E75CE552D880E754C0
:10499000E552D880E7545FD9030EDB50010B0BE1E1
:1049A000080EDB5008E0B2D801E08DD0080EDB50D5
:1049B000BED8080EDB6A170EDB5007E088D9170E49
:1049C000F1D903E1151C01E17ED0160EDB5016E093
:1049D0007ED9300EE66E9FD802E1151C74E077D9BF
:1049E000DFCFE6FF8AEC35F0E552E552E552F4CF31
:1049F00015F00001F31C02E1151C65E0050EDBCF8C
:104A000014F0160EDB50D880145409E2050EDBCFEB
:104A1000E7FF160EDB50E75E050EE7CFDBFF300E3B
:104A2000E66E050ECBD94FE1390EDB2ADBCFE9FF6D
:104A30003A0E01E3DB2ADBCFEAFF090EEFCFDBFF03
:104A4000DB500EE044D9090EADD902E1151C3BE064
:104A5000390EDB2ADBCFE9FF3A0EEDE3DB2AEBD799
:104A600055D831E1160EDBCFE6FF080EC3D8E5526C
:104A7000E7245DD82ED0070EDB50030A1CE0010AA4
:104A800014E0030A07E07BD9DBCFEEFF020EDBCF99
:104A9000EDFF1FD0F5D8196A17AE02D01868196853
:104AA0002CD8BCD819C0EEFF14D0EAD817BE1868AD
:104AB00024D8B4D80ED063D9DBCFEFFF0AD07BD98E
:104AC00005E1151C03E1F368F46810D0FCD801E39C
:104AD000DB2A79D908EF21F0010EDBCF14F0020EAA
:104AE000DBCF15F014C0F3FF15C0F4FF3B0EE15C03
:104AF00002E2E16AE552E16ECBD029D9020E6EEFF7
:104B000026F061D90800F550DF6E1200200EE66E27
:104B1000080EDEEF26F08AEC35F0E552E552E5525C
:104B2000F3CF14F0F4CF15F00001F31C1200146E53
:104B3000156AD950010F4DD91450EE261550ED22AB
:104B40001200185E000E195AF70E18C0DBFFF80E9F
:104B500019C0DBFF18C0E9FF19C0EAFF1200DBCF64
:104B6000F4FFF350F45C1200DB50E76E040EE7CF65
:104B7000DBFF12000A0EDBCF14F00B0EDBCF15F0BB
:104B80000C0EDBCF16F00D0EDBCF17F01450151006
:104B9000161017101200130EEECFDBFF140EEDCF20
:104BA000DBFF130EDBCF14F0140EDBCF15F000018A
:104BB000800E15141200F70EDBCF18F0F80EDBCFC5
:104BC00019F01200050EDB50E66ED950130F01D913
:104BD000E552E750EE6EED6A12000A0EDBCF06F0EA
:104BE0000B0EDBCF07F00C0EDBCF08F00D0EDBCF8A
:104BF00009F01200DBCFE6FF150EDBCFE6FF050E56
:104C0000DB50E552E724E552E7241200DB50CED812
:104C1000010EF36E060EF3CFDBFF1200EE50EFCF66
:104C2000EAFFE96E16C0EEFF17C0EEFF18C0EEFFF8
:104C30001200D9CFE6FFDACFE6FFE1CFD9FFE2CF0E
:104C4000DAFF1200DFCFE6FFE66ACFEC17F0E5529D
:104C5000E552F3501200E76E080EE7CFDBFF1200BB
:104C6000EECF14F0EECF15F0EFCF16F0176A12006A
:104C7000050EDBCF14F0150EDB50D8801454120053
:104C8000010EDBCF16F0020EDBCF17F0186A120010
:104C9000E552E5CFDAFFE7CFD9FF12000A0E14C0C4
:104CA000DBFF0B0E15C0DBFF1200D9500A0FE9EF36
:104CB00026F0F36E070EF3CFDBFF1200EECF14F0F9
:104CC000EFCF15F01200010EDB2A020E1200FC0ECF
:104CD000DBCFE6FFFD0EDBCFE6FF1200145E000E19
:104CE000155AF70E14C0DBFFF80E15C0DBFF14C019
:104CF000E9FF15C0EAFF1200DA20EA6EEF2AEECFD4
:104D0000F6FF000EEF22EECFF7FFEF22EECFF8FF17
:104D10001200040EDBCFE6FF130EDB50E552E75C1A
:104D20009ADFDB5004DF060EDB501200090EDB5069
:104D30000A0DF350DF24D00FE76E090EE7CFDBFF3B
:104D400081EF25F0DB50F36E050EAFEF25F0F70E87
:104D5000DBCF14F0F80EDBCF15F01200DFCFE6FF4B
:104D60008BEF25F028DF030EECDE30EF26F0DDECD4
:104D700020F0E552E552E552E55200091200BDDE91
:104D8000EE50EFCFEAFFE96E010E1200130EDB507A
:104D9000F36E040EAFEF25F0040EDB50F36E090E38
:104DA000AFEF25F0DBCFE6FF8BEF25F0E76E050ECA
:104DB000E7CFDBFF12008BDFAEEF26F0DBCFE6FFA5
:104DC00086DFB7EF26F0D950F90FE96EFF0E7CEFC2
:0C4DD00026F0E96E000EDA20EA6E1200F8
:044DDC0028632920FF
:104DE000436F707972696768742053696572726184
:104DF00020526164696F2053797374656D732C2040
:104E00004C4C4300012A3101016801010101012DCF
:104E100001010101010101680101012201010101FA
:104E20000101010101010101680101012D01012AB6
:104E300073616A293F3E3C3830202123272F01012E
:104E40000131014C560611150902140B10041E0DF8
:104E50001207050F161B0A08030C180E191D130163
:104E6000010122010CCF2A1E00000000000CB11F1E
:104E70001E00000000000CCF2A0A00000CB11F1E0B
:104E800000000000000CCF2A0A00000CCF2A0A0004
:104E9000000CCF2A1E000000000010B11F100000FF
:104EA00010B11F1E000000000010B11F1000001004
:104EB000B11F1E000010B11F10000010B11F1E0016
:104EC0000000000014B11F14000014B11F1E0000E8
:104ED00000000014B11F14000014B11F1E000014C4
:104EE000B11F14000014B11F1E0000000000109537
:104EF0000C10000010950C1E000000000010B11FE7
:104F000010000010B11F1E000000000010950C10D2
:104F1000000010950C1E000010950C10000010955C
:104F20000C1E000000000010B11F10000010B11F87
:104F30001E000010B11F10000010B11F1E00000065
:104F4000000010950C10000010950C10000010953A
:104F50000C1E000000000010B11F10000010B11F57
:104F600010000010B11F1E00000000000C45121EB2
:104F700000000000000CCF2A0A00000C45121E00A1
:104F800000000000000000145A12140000145A120D
:104F9000140000145A12C80000C800000001006488
:104FA000BB0F645A1200010014AB181E0000000071
:104FB000001406231E0000000000102D0910000040
:104FC000102D091E000000000010890B10000010B9
:104FD000890B1E0000000000C82D09000100C889CF
:104FE0000B000100102D09100000102D0910000009
:104FF000102D091E000000000010890B1000001089
:10500000890B10000010890B1E0000000000649541
:105010000C64000000010064411064000000010005
:10502000C8E71800010014E71814000014E7183C42
:1050300000000001000AE7184600000001000AE72E
:10504000180A00000AE7189600000001000AE71895
:105050001E00000001000AE7180A00000AE7181EF7
:1050600000000001000AE7183200000001000AE712
:10507000180A00000AE7183200000001000AE718C9
:105080001E00000AE7183200000001000AE7182895
:1050900000000001000A912C0A00000A912C0A006D
:1050A000000A912C0A00000A912C0A00000A912C97
:1050B0000A00000000000A0D370A00000A0D370A36
:1050C00000000A0D370A00000A0D370A00000A0D19
:1050D000370A0000000000140D3714912C140D370E
:1050E00014912C140D3714912C140D3714912C1489
:1050F0000D3714912C000000000000140D3714919E
:105100002C140D3714912C140D3714912C140D37C9
:1051100014912C140D3714912C140D3714912C1458
:105120000D3714912C140D37000000000000149569
:105130000C14000014950C14000014950C140000BD
:1051400014950C14000014950C14000000000014B9
:105150006B0E140000146B0E140000146B0E140080
:1051600000146B0E140000146B0E140000000000FD
:1051700014950C146B0E14950C146B0E14950C14E2
:105180006B0E14950C146B0E14950C146B0E000022
:1051900000C87C0A00010020950C10000010950C3E
:1051A0001E000000000010000020B11F30000000B1
:1051B000000027F9140D00000DF91427000027F94D
:1051C000140D000027F9140D000027F91427000022
:1051D0000000000DF9142700000DF9140D00002740
:1051E000F9140D00000DF9142700000DF9140D003D
:1051F0000027F9140D00000DF9142700000000002D
:1052000027F9140D00000DF9142700000DF9140DF5
:10521000000027F9142700000000000C59190CB1F8
:105220001F0C0A261E00000000000CB11F0A00001F
:105230000CCF2A1E0000000000844F000000000078
:1052400030001830003030004830006030007830D6
:1052500000903000A83000C03000D83000F030009E
:1052600008310020310038310050310068310080B1
:105270003100983100B03100C83100E03100F83120
:1052800000103200283200403200583200703200E4
:10529000883200A03200B83200D03200E832006418
:1052A0004E00000000764E000000006C4F00000031
:1052B000009A4E000000006D4E00000000874F0075
:1052C0000000009F4F00000000A84F00B14F00BA3F
:1052D0004F00C94F00D84F00DE4F000E500017504E
:1052E00000754F0000000020500000000026500014
:1052F0000000003550000000003E5000000000A9F2
:105300004E00000000955000B650002E51004F5145
:1053100000E44F00F94F00854E000000009151005D
:105320000000004D5000000000565000000000C476
:105330004E00000000D34E00000000EE4E00FD4E77
:10534000000C4F00274F00424F00574F009751006D
:10535000A651006550000000006E5000000000D70C
:1053600050000000007051000000007D500000005F
:1053700000B25100000000D351000000008C50002A
:10538000000000005200000000FB50000000001B65
:1053900052000000002A5200000000080C101418EF
:0353A0002028645E
:0C53A4009D989D9ACAD80001E86B949C6B
:1053B000948E9F9A9F98240EAC6E900EAB6EB8861A
:1053C000800EE66E250EE66EE66AE66A3AD85FEF74
:1053D0002BF09D989D9AAB9E120061D9186A2D0EF4
:1053E000196E310E1A6E010E1B6E18C006F019C030
:1053F00007F01AC008F0096EFB0EDBCF0BF0FC0EB5
:10540000DBCF0CF0FD0EDBCF0DF0FE0EDBCF0EF090
:1054100004EC36F006C014F007C015F008C016F012
:1054200009C017F01406000E155A165A175AD890CC
:10543000173216321532143214C0F3FF15C0F4FFC0
:1054400033D12DD9030EE126D950FB0FE96EFF0EA3
:10545000DA20EA6EEECFE6FFEECFE6FFEECFE6FF14
:10546000EFCFE6FFBADF2BD9F3CFDEFFF4CFDDFFBE
:105470009D50200B03E19D50100B06E0010EF36ED2
:10548000020EF3CFDBFF02D0020EDB6A9D989D9ADD
:10549000DECF14F0DDCF15F015C014F0156A1450EE
:1054A000B06EDF50AF6E020EDB5002E09D889D8A29
:1054B000030EE15C02E2E16AE552E16EF5D09E5036
:1054C000100B05E09D50100B02E00AD8010C9E5015
:1054D000200B05E09D50200B02E010D8010C000CC1
:1054E000DED8E65207D976D8E552E552000903E046
:1054F000DF50AD6E01D09D98E552D6D0D0D8E6529F
:10550000ABA203D0AB98AB880BD0AE50DF6EABB480
:1055100007D0DFCFE6FFF30EE66E000EDDD802D037
:105520000001E881E552C0D0EAD801E1000C010C8D
:10553000E6D803E1F251010B01E1000C010C320E3F
:10554000E66E000EE66E030EE66EF30EE66E000EDD
:10555000BBD8640EE66E000EE66E0F0EE66EED0E24
:10556000E66E000E64EF2BF09AD89D9AA1D8F30E48
:10557000E66E000EE66E07EC34F0A1D8000903E0F9
:105580009D8A010E02D09D8A000E8ED088D800011F
:10559000F8B113D0F751EA6AF325E96EF451EA2223
:1055A000EF50E66EFD0EDBCFE9FFFE0EDBCFEAFF2C
:1055B000E552E750EF6E010E01D0000E75D06FD8A6
:1055C0009D98FE0EDBCFE6FFED0EE66E000E84D852
:1055D0009D886AD064D86CD8ED0EE66E000EE66E3B
:1055E00007EC34F06CD860D05AD889D80DE17BD85C
:1055F0005FD834EC2CF0E552E552F3CFEBF0F4CF6A
:10560000ECF013D8010E01D0000E4ED048D877D858
:105610000AE169D8FB0EDBCFEBF0FC0EDBCFECF040
:1056200004D8010E01D0000E3FD069D81BE0EB5129
:10563000EC1113E0F251020B10E1E9C0E9FFEAC0FE
:10564000EAFFE92B000EEA23EF50E66EB8DFE552E1
:105650000001EB07000EEC5BEAD7EB51EC1102E125
:10566000E96BEA6B12000001E96BEA6B9FEF2AF02D
:1056700016D8E6520001F8B110D03CD887DFE552C9
:10568000E552DFCFE6FF2EEC01F0E552000905E11F
:1056900031D86ADFE552E552EDD7E55205D0D9CFD2
:1056A000E6FFE1CFD9FF1200E552E7CFD9FF1200A4
:1056B000FD0EDBCFE6FFFE0EDBCFE6FF1200E5526C
:1056C000E552E552E5521200E66ED1EC33F0146E6D
:1056D000050EE15E14501200E66EEBEC33F0E5527D
:1056E000E552E5521200FD0EDBCFE9F0FE0EDBCFF6
:1056F000EAF01200D9CFE6FFDACFE6FF1200000190
:06570000E951EA1112005C
:0A570600D9CFE6FFDACFE6FFFA0E76
:10571000E3CFD9FFFB0EE3CFDAFFFC0EE3CFE9FFC7
:10572000FD0EE3CFEAFFE9CFF3FFEACFF4FFF80E77
:10573000E35003E1F90EE35008E0F80EE30602E25D
:10574000F90EE306DECFEEFFF2D7FF0EE3CFDAFF6E
:10575000E552FF0EE3CFD9FFE5521200D9CFE6FFA5
:10576000DACFE6FFFA0EE3CFD9FFFB0EE3CFDAFF85
:10577000FC0EE3CFE9FFFD0EE3CFEAFFE9CFF3FF35
:10578000EACFF4FFE950D95CEA50DA580EE3F80E9C
:10579000E35003E1F90EE35024E0F80EE30602E2E1
:1057A000F90EE306DECFEEFFF2D7F80EE350D9266E
:1057B000F90EE350DA22DD52F80EE350E926F90E35
:1057C000E350EA22ED52F80EE35003E1F90EE35004
:1057D00008E0F80EE30602E2F90EE306DDCFEDFF86
:1057E000F2D7FF0EE3CFDAFFE552FF0EE3CFD9FF8A
:1057F000E5521200D9CFE6FFDACFE6FFFA0EE3CF8B
:10580000D9FFFB0EE3CFDAFFFC0EE3CFE9FFFD0E7D
:10581000E3CFEAFFE9CFF3FFEACFF4FFDECFEFFFFC
:10582000EE66FCD7FF0EE3CFDAFFE552FF0EE3CFC3
:10583000D9FFE5521200FB0EE3CFF6FFFC0EE3CFDB
:10584000F7FFFD0EE3CFF8FFFE0EE3CFE9FFFF0EFB
:10585000E3CFEAFFE9CFF3FFEACFF4FF0900F5CF8A
:10586000EFFFEE66FBD71200FE0EE3CFE9FFFF0E5F
:10587000E3CFEAFFF36AF46AEE5203E0F34AF42A54
:10588000FBD71200FF0EE3CFF8FFE552FF0EE3CF88
:10589000F7FFE552FF0EE3CFF6FFE552E66AE66A50
:1058A000E66A0900F55209E0FD0EE32A05E1FE0E65
:1058B000E32A02E1FF0EE32AF4D7FD0EE3CF07F05F
:1058C000FE0EE3CF08F0FF0EE3CF09F01200D9CFB0
:1058D000E6FFDACFE6FFFA0EE3CFD9FFFB0EE3CF08
:1058E000DAFFFC0EE3CFE9FFFD0EE3CFEAFFE9CFDD
:1058F000F3FFEACFF4FFF80EE35003E1F90EE350B3
:105900000BE0F80EE30602E2F90EE306DECFEFFF4E
:10591000EE66F1D7DD52EFD7FF0EE3CFDAFFE552A7
:10592000FF0EE3CFD9FFE5521200FB0EE3CFF6FFE7
:10593000FC0EE3CFF7FFFD0EE3CFF8FFFE0EE3CF43
:10594000E9FFFF0EE3CFEAFFE9CFF3FFEACFF4FF71
:10595000F90EE35003E1FA0EE3500CE0F90EE30612
:1059600002E2FA0EE3060900F5CFEFFFEE66F0D78C
:105970000A00EED71200FE0EE3CFE9FFFF0EE3CFE1
:10598000EAFFF36AF46AFD0EE350EF5C04E1E9CF4D
:0C599000F3FFEACFF4FFEE66F6D712003A
:04599C009EB09DA07C
:1059A00001D002D0000E12000E01F6CF1FFEF7CF7D
:1059B00020FEF8CF21FEF5CF22FEF3CF23FEF4CF59
:1059C00024FEE9CF25FEEACF26FED9CF27FEDACF87
:1059D00028FE550EF29ECE5C2D6FC30ECF5A2DCEF3
:1059E000CEFFF28E296729072A672A072B672B0724
:1059F0002C672C073C673C073D673D073E673E0729
:105A00005C675C07352F02D0140E356F3F2F07D02F
:105A1000C80E3F6FE86A402B41234223432336A13F
:105A20002CD029672AD036A505D037CE29FE119D66
:105A3000369523D0466711D044CEE9FF45CEEAFF24
:105A4000EFCF46FE466701D017D0444B452B010EE1
:105A5000466303D03ACE29FE10D0D890463309E0F1
:105A600003E237CE29FE02D039CE29FE118D3685CC
:105A700004D038CE29FE01D0369136A93CD02A6711
:105A80003AD047CEE9FF48CEEAFF030E4727E86A3F
:105A90004823EE5027E02A6FEECF2FFEEE50306FF6
:105AA00003E12F5101E11CD05B5110E02F3530355F
:105AB0009D0D5751F402F336F43406E2F336E83420
:105AC00003E2F336E83403E3FF0E01D057519D9211
:105AD0001A6F2FCE12FE30CE13FE9D8211810BD095
:105AE000119109D0EE5005E04FCE47FE50CE48FE52
:105AF00002D03699119136AB3CD02B673AD049CEC3
:105B0000E9FF4ACEEAFF030E4927E86A4A23EE502E
:105B100027E02B6FEECF31FEEE50326F03E13151B3
:105B200001E11CD05B5110E0313532359D0D5851EB
:105B3000F402F336F43406E2F336E83403E2F336E3
:105B4000E83403E3FF0E01D058519D921B6F31CE14
:105B500014FE32CE15FE9D8211850BD0119509D011
:105B6000EE5005E051CE49FE52CE4AFE02D0369BA1
:105B7000119536AD3CD02C673AD04BCEE9FF4CCED8
:105B8000EAFF030E4B27E86A4C23EE5027E02C6F08
:105B9000EECF33FEEE50346F03E1335101E11CD000
:105BA0005B5110E0333534359D0D5951F402F33615
:105BB000F43406E2F336E83403E2F336E83403E380
:105BC000FF0E01D059519D921C6F33CE16FE34CE7C
:105BD00017FE9D8211890BD0119909D0EE5005E076
:105BE00053CE4BFE54CE4CFE02D0369D119928CE9A
:105BF000DAFF27CED9FF26CEEAFF25CEE9FF24CE55
:105C0000F4FF23CEF3FF22CEF5FF21CEF8FF20CE06
:0C5C1000F7FF1FCEF6FF9E90010E120061
:045C1C0027D9E6524C
:105C200094869488160EC66E010EC56EFE0EDB506D
:105C3000E824C86EC76AFC0EDBCFDFF2FD0EDBCFB7
:105C4000E0F2FA0EDBCFE1F2FB0EDBCFE2F2F90E6F
:105C5000DB040201E36FF70EDBCFE4F2F80EDBCFDB
:105C6000E5F2F50EDBCFE6F2F60EDBCFE7F2C68A01
:105C70009E96E552E552E7CFD9FF1200F7D8020E03
:105C8000E126010EDB6A9EA648D0C69C2D0EC714E5
:105C9000090A1EE0050A02E0010A37E1C950DF6E79
:105CA0009E96E4C2E6FFE5C2E6FFE6C2E9FFE7C270
:105CB000EAFFEF50E66E3AD8E552E552E552DF6E64
:105CC000E6C2E9FFE7C2EAFFEF6ADF5017E11AD048
:105CD000C950DF6E9E96C688E3C2E6FFDFC2E6FFCC
:105CE000E0C2E6FFE1C2E6FFE2C2E6FF5AD8146E68
:105CF000050EE15E1450DF6EDF5004E0010EDFCFD1
:105D0000DBFF0BD0010EDB6808D0C950DF6E9E961A
:105D1000C69CC688DE52050EDD6E010EDB50146E89
:105D2000020EE15C02E2E16AE55291D09FD8030ED7
:105D3000E1260E013C69FE0EDB50C96E9E96C688B8
:105D4000FC0EDBCF08F0FD0E88D8FE0EDB50DF6EB8
:105D5000DF501FE09E50080B02E13C51FBE13C513B
:105D600002E1010E17D02D0EC7142C0A07E0040A19
:105D700004E09E96C688020E0DD0DF6ADF5005E073
:105D80007AD801E3DB2AEF50C96E9E96C688DF06FB
:105D9000DFD7000E146E030EE15C02E2E16AE55209
:105DA00056D064D8050EE1260E013C696CD8EF6A26
:105DB0009E50080B02E13C51FBE13C512BE02D0EC3
:105DC000C714290A2DE1040EC9CFDBFF9E96C688B1
:105DD000FB0EDBCF08F0FC0E40D8040EDB50F36E58
:105DE000FA0EDBCFF4FFF350F45C06E2FA0EDB5060
:105DF000E76E040EE7CFDBFF040EDB50DF6EDF50F3
:105E00001EE09E50080B03E10E013C51FAE10E0129
:105E10003C5102E1010E14D02D0EC714290A04E0F2
:105E20009E96C688020E0CD09E96C68824D801E3A2
:105E3000DB2AC9CFEFFF27D8EF2ADF06E0D7000E15
:105E4000146E050EE15C02E2E16AE55200D0E16EFB
:105E50001450E552E7CFD9FF1200DBCF09F0DE5234
:105E600008C0DEFF09C0DDFFDD521200D9CFE6FF1A
:105E7000E1CFD9FF1200010EDBCFE9FFDB2A020ED2
:105E8000DBCFEAFF1200FD0EDBCFE9FFFE0EDBCF1A
:045E9000EAFF120013
:0C5E940040771B0080841E00A025260023
:105EA000A0252600E067350000093D00404B4C006E
:105EB000404B4C004456510044565100C49451008C
:105EC000C4945100E4E25100E4E251006CF6510048
:105ED000AE0452006C7352006C735200C0CF6A0063
:105EE000A0636F008096980080969800201D9A000D
:105EF00070E09A00809FD500B0F6DA00C0E1E400BF
:105F0000C0E1E40020B21301C0381501406F400128
:105F1000104D470190CA7B0130517D01003FAB011C
:105F2000A02FC50180F0FA0280F9370300449508DC
:105F3000004DD2080007AE09F050B00980733B0D48
:105F4000403A690D00B108198074D21A806DC335CA
:105F50000028503700E6E849006D7C4D0000000045
:105F60000000000000000000000000000000000031
:105F70000000000000000000000000000000000021
:105F80000000000000000000000000000000000011
:105F900000000000A0252600A0252600E0673500AF
:105FA00080EE3600404B4C00404B4C00C0CF6A00A6
:105FB00008B86C008096980080969800201D9A0082
:105FC00070E09A00809FD50070E9D700C0E1E4003E
:105FD000C0E1E40020B2130130561401406F4001CB
:105FE000807C430190CA7B01D0667C01003FAB01FD
:105FF000E0D2AF0180F0FA022077FC02004495085D
:10600000A0CA96080007AE09F050B00900000000D1
:106010000000000000000000000000000000000080
:106020000000000000000000000000000000000070
:106030000000000000000000000000000000000060
:106040000000000000000000000000000000000050
:106050000000000000000000000000000000000040
:106060000000000000000000000000000000000030
:106070000000000000000000000000000000000020
:106080000000000000000000000000000000000010
:04609000000000000C
:0C6094000E01F6CF00FEF7CF01FEF8CFA2
:1060A00002FEF5CF03FEF3CF04FEF4CF05FE0E6B28
:1060B000106B12510627135107231451082715514D
:1060C000092311B101D027D011A305D01ECE0EFE99
:1060D00007BF0E6D18D0000EF86E0751E846E8466F
:1060E00006BFE88206BDE88007BDE86CF66ECA0E02
:1060F000F626680EF76E02E3F74AF82A0800F55014
:1061000007BFE86C0E6F1A510E030EBFF45EF3CF9B
:1061100010FEF4CF0EFE11A527D011A705D01ECE7C
:106120000FFE09BF0F6D18D0000EF86E0951E8463A
:10613000E84608BFE88208BDE88009BDE86CF66E55
:10614000CA0EF626680EF76E02E3F74AF82A080030
:10615000F55009BFE86C0F6F1B510F030FBFF45EC2
:10616000F3501027F4500E231051800FE86A0E23CD
:10617000800E0E25BE6E0E6B106B16510A2717513E
:106180000B2318510C2719510D2311B901D027D019
:1061900011AB05D01ECE0EFE0BBF0E6D18D0000E3B
:1061A000F86E0B51E846E8460ABFE8820ABDE8806F
:1061B0000BBDE86CF66ECA0EF626680EF76E02E3AB
:1061C000F74AF82A0800F5500BBFE86C0E6F1C5117
:1061D0000E030EBFF45EF3CF10FEF4CF0EFE11AD32
:1061E00027D011AF05D01ECE0FFE0DBF0F6D18D0FA
:1061F000000EF86E0D51E846E8460CBFE8820CBD73
:10620000E8800DBDE86CF66ECA0EF626680EF76ED5
:1062100002E3F74AF82A0800F5500DBFE86C0F6F4B
:106220001D510F030FBFF45EF3501027F4500E23DF
:106230001051800FE86A0E23800E0E25BB6E9E92D1
:1062400005CEF4FF04CEF3FF03CEF5FF02CEF8FF38
:0A62500001CEF7FF00CEF6FF1200AA
:06625A00FF0EE3CFEAFF96
:10626000E552FF0EE3CFE9FFE552E66AE66AE66A29
:10627000E66AD9CFE6FFDACFE6FFFA0EE124D96E5F
:10628000FF0EE220DA6EE66AE66AE66AE66AE66A27
:10629000200EEF5C06E0090EEF5C03E0EF6603D032
:1062A0006BD0EE50F5D72D0EEF5C03E1FF0EE32A25
:1062B00003D02B0EEF5C01E1EE502F0EEF6444D0C3
:1062C0003A0EEF6041D0D890F50EE336F60EE33685
:1062D000F70EE336F80EE336FB0EDECFE3FFFC0EDF
:1062E000DECFE3FFFD0EDECFE3FFFE0EDDCFE3FFEB
:1062F000DD52DD52D890F50EE336F60EE336F70E9A
:10630000E336F80EE336D890F50EE336F60EE336B4
:10631000F70EE336F80EE336FB0EE350DE26FC0EF6
:10632000E350DE22FD0EE350DE22FE0EE350DD22BE
:10633000DD52DD52300EEE5CDE26000EDE22DE2265
:10634000DD22DD52DD52B9D7FF0EE3CFE8FFE85280
:1063500013E0F50EE31EF60EE31EF70EE31EF80E35
:10636000E31EF50EE32A08E1F60EE32A05E1F70E37
:10637000E32A02E1F80EE32AE552E552E552E5523E
:10638000E552D9CFE9FFDACFEAFFEECF06F0EECF44
:1063900007F0EECF08F0EFCF09F0FF0EE3CFDAFF02
:1063A000E552FF0EE3CFD9FFE552E552E552120068
:1063B000006AE86A0EAEE5EF31F00B6C0C1E0D1EA4
:1063C0000E1E0C220D220E22001E09AEF0EF31F03F
:1063D000066C071E081E091E072208220922001E3D
:1063E00004EC36F009BE07EF32F000AE000C066C8C
:1063F000071E081E091EE86A072208220922026CED
:10640000031E041E051E032204220522000C00BEEA
:10641000F7EF31F00188FF0C09C013F008C012F04B
:1064200007C011F007500C02F4CF05F0F3CF04F0D1
:1064300008500D02F4CF07F0F3CF06F00C02F35032
:106440000526F4500622E86A072211500D02F35087
:106450000526F4500622E86A072209500C02F35080
:106460000626F450072209500D02086AE86A08223D
:10647000F3500726F450082211500E02F35006265E
:10648000F4500722096AE86A0822092212500E0213
:10649000F3500726F4500822E86A092213500E022E
:1064A000F3500826F4500922000C09C013F008C06C
:1064B00012F008500D02F4CF07F0F3CF06F00950A8
:1064C0000E02F4CF09F0F3CF08F00D02F3500726C7
:1064D000F4500822E86A092212500E02F3500726EF
:1064E000F4500822E86A09220EAE7BEF32F0125017
:1064F000085E1350095A13AE000C0D50085E0E5082
:04650000095A000C28
:0C6504008DD8F8CFE4FFF5CFE4FFE6529D
:106510004AEC30F0E552E5CFF5FFE5CFF8FF8ED03D
:106520007FD8F6CFE4FFF7CFE4FFF8CFE4FFF5CF55
:10653000E4FFF3CFE4FFF4CFE4FFFACFE4FFFBCFB7
:10654000E4FF00EE00F0140EE80403E3EECFE4FFF6
:10655000FBD700EE14F0120EE80403E3EECFE4FFE5
:10656000FBD7E6525FEC2AF0000902E1CEEC2CF0FA
:10657000E55200EE25F0120EE80403E3E5CFEDFF4F
:10658000FBD700EE13F0140EE80403E3E5CFEDFFB4
:10659000FBD7E5CFFBFFE5CFFAFFE5CFF4FFE5CF73
:1065A000F3FFE5CFF5FFE5CFF8FFE5CFF7FFE5CF48
:1065B000F6FF44D0D9CFE6FFE1CFD9FF240EE12684
:1065C00084EC11F09D829D80F28EF28C0E01010E02
:1065D0003B6F9D889D8A0400F5EC15F0146814C08B
:1065E000E6FF3EEC2EF0E552E7CF14F0DF6E145CD0
:1065F00002E17CEC12F00CEC1AF08BEC1AF015ECCA
:106600002BF038EC2BF030EC00F0E5D7240EE15CF9
:1066100002E2E16AE552E16EE552E7CFD9FF1200EE
:10662000D8CFE4FFE0CFE4FFE46EDACFE4FFE2CFBF
:10663000DAFFE9CFE4FFEACFE4FF1200E5CFEAFF9B
:10664000E5CFE9FFE5CFDAFFE550E5CFE0FFE5CFA5
:04665000D8FF10005F
:0C665400D9CFE6FFE1CFD9FF020EE1260E
:106660000001F96BFA6BFB6BFC6BD950FC0FE96E08
:10667000FF0EDA20EA6EEFCFF6FF020EEE26EFCF26
:10668000F7FF000EEE22EFCFF8FF000EEE2209001A
:10669000F5CFFBF00A00F5CFFCF0FA0EDB06FB0E9F
:1066A00001E2DB06FA0EDBCF14F0DB06FB0EDBCFDC
:1066B00015F001E2DB06145015103FE00400D9503C
:1066C000FC0FE96EFF0EDA20EA6EEFCFF6FF020E46
:1066D000EE26EFCFF7FF000EEE22EFCFF8FF000E11
:1066E000EE220900F5CFF9F00A00F5CFFAF0100E0E
:1066F000DE6EDD6AD9CFE9FFDACFEAFFEE50ED10AA
:106700001BE00001FB51800B0CE00001D890F93731
:10671000FA37FB37FC37210E0001FB1B0001FC7729
:1067200006D00001D890F937FA37FB37FC37DF067F
:10673000010E01E2DB06DED7B5D7200EDE6EDD6A84
:10674000D9CFE9FFDACFEAFFEE50ED101BE00001F0
:10675000FB51800B0CE00001D890F937FA37FB377A
:10676000FC37210E0001FB1B0001FC7706D0000165
:10677000D890F937FA37FB37FC37DF06010E01E214
:10678000DB06DED7FBC0F3FFFCC0F4FF00D0020E37
:10679000E15C02E2E16AE552E16EE552E7CFD9FF42
:0267A0001200E5
:0E67A200D9CFE6FFE1CFD9FF55D8FB0EDBCFF4
:1067B000EEFFFC0EDBCFEDFF4ED8020E53D8FA0EE3
:1067C000DBCFEFFF60D8EF925ED8EF8060D8EF6A42
:1067D00062D8EF6A54D072D8020B17E158D867D844
:1067E000FC0EDBCFEFFF4FD8EF9051D858D802E323
:1067F0004ED8EF6A4CD8EFCF14F04DD8EF50145C60
:1068000002E141D8EF82010E01D0000E38D056D8F7
:10681000010B1FE140D84BD8EF50E66EFB0EDBCFEB
:10682000E9FFFC0EDBCFEAFFE552E750EF6E2BD815
:10683000EF9231D834D802E32ED8EF6A2CD8EFCFBC
:1068400014F025D8EF50145C02E11DD8EF80010E42
:1068500001D0000E14D0FD0EDBCFE9FFFE0EDBCF22
:10686000EAFF1200E926000EEA2212001450EE247C
:10687000E76E1550EE20EA6EE7CFE9FF1200E55211
:10688000E7CFD9FF1200E7DF050E32EF34F0E3DF88
:10689000030E32EF34F0DFDF040E32EF34F0EFCFCF
:1068A00014F0D9DF020EDEDFEF50145C1200EF505F
:1068B000EF2A146E156ACFDF36EF34F0D9CFE6FF3A
:0A68C000E1CFD9FFE0DFEF50120036
:0668CA00000102020304BC
:1068D000050506070809090A0B0C0C0D0E0F101010
:1068E00011121313141516161718191A1A1B1C1D3A
:1068F0001D1E1F2020212223232425262627282968
:10690000292A2B2C2C2D2E2E2F303131323333349B
:10691000353636373838393A3A3B3C3D3D3E3F3FD5
:106920004041414243434445454647474848494A18
:106930004A4B4C4C4D4E4E4F4F5051515252535466
:10694000545555565657585859595A5A5B5B5C5DC1
:106950005D5E5E5F5F606061616262636364646527
:10696000656666666767686869696A6A6A6B6B6CA0
:106970006C6D6D6D6E6E6F6F6F7070707171717226
:1069800072727373737474747575757676767677C0
:10699000777778787878797979797A7A7A7A7A7B68
:1069A0007B7B7B7B7C7C7C7C7C7C7D7D7D7D7D7D25
:1069B0007D7E7E7E7E7E7E7E7E7E7E7E7F7F7F7FF4
:0A69C0007F7F7F7F7F7F7F7F7F7FD7
:0669CA00D9CFE6FFDACF91
:1069D000E6FFE1CFD9FFE2CFDAFFE652E652E65218
:1069E000E652D950F90F146EFF0EDA20156E020E22
:1069F00014C0DBFF030E15C0DBFF020EDBCFE6FF8A
:106A0000030EDBCFE6FFF90EDBCFE6FFFA0EDBCF9E
:106A1000E6FFFB0EDBCFE6FFD950FC0FE66EFF0E64
:106A2000DA20E66EF3EC20F0146E070EE15C02E271
:106A3000E16AE552E16E1450F3CFDEFFF4CFDDFFE3
:106A4000FC0EDBCFE9FFFD0EDBCFEAFFEF6ADECF06
:106A500014F0DDCF15F014C0F3FF15C0F4FF040EE1
:106A6000E15C02E2E16AE552E16EE552E5CFDAFF70
:066A7000E7CFD9FF120080
:0A6A76002A0EF66E000EF76E000EF9
:106A8000F86E0F010900F550696F0900F5506A6F43
:106A900003E1696701D03DD00900F550646F09003A
:106AA000F550656F0900F550666F09000900F55053
:106AB000E96E0900F550EA6E090009000900F55079
:106AC000676F0900F550686F09000900F6CF6BFF8A
:106AD000F7CF6CFFF8CF6DFF64CFF6FF65CFF7FF00
:106AE00066CFF8FF0F01675302E1685307E0090022
:106AF000F550EE6E6707F8E26807F9D76BCFF6FF3F
:106B00006CCFF7FF6DCFF8FF0F016907000E6A5BCE
:046B1000BFD71200D9
:0C6B1400D9CFE6FFDACFE6FFE1CFD9FFD2
:106B2000E2CFDAFFFB0EDBCF14F0FC0EDBCF15F06B
:106B30000001800E15141AE1FB0EDBCFE9FFFC0EFD
:106B4000DBCFEAFFEECFF3FFEDCFF4FFEE2A000E2E
:106B5000EF22F3CFE9FFF4CFEAFFFD0EDBCFEFFF2B
:106B6000EF50156AF36E15C0F4FF10D0FB0EDB502A
:106B7000FE0806E1FD0EDBCFE6FF85EC36F005D022
:106B8000FD0EDBCFE6FFFFEC17F0E552E552E5CF57
:086B9000DAFFE7CFD9FF120084
:086B980006500B02F3CF02F0DE
:106BA000F4CF03F00C02F3500326000EF420046E21
:106BB00006500D02F3500426000EF420056E065018
:106BC0000E02F350052607500B02F3500326F45033
:106BD0000422000E052207500C02F3500426F45044
:106BE000052207500D02F350052608500B02F35002
:106BF0000426F450052208500C02F35005260950D3
:086C00000B02F35005261200FF
:086C0800056A046A036A026ACE
:106C1000200EE76ED890063607360836093602365B
:106C20000336043605360B50025C0C5003580D50E9
:106C300004580E50055809E30B50025E0C50035ADD
:106C40000D50045A0E50055A062AE72EE4D71200BA
:106C5000202073727330303938762000206E6F2018
:106C600069642073657420007031007030007430E6
:106C7000300074253264006F332530356C64006F4A
:0F6C800032006F31006F3000662530356C6400D4
:106C9000FF0EE350276EEF0E01D0F30EE76EE72EE6
:106CA0004FEF36F00C0E266EE76AE72E55EF36F002
:0E6CB000262E54EF36F0272E4DEF36F0120050
:026CBE00056A65
:106CC000046A100EE76ED890083609360436053689
:106CD0000D50045C0E50055805E30D50045E0E5037
:0A6CE000055A082AE72EF0D712002B
:066CEA001DEE00F02DEE8E
:106CF00000F0F86A019CA1EC36F03BEC35F0A8EC12
:0A6D000036F0DAEC32F0FBD7120097
:066D0A00FF0EE350ACBADD
:106D100004D0AF6AAB8EAC8A949CACA2FED7AD6EA9
:066D2000F36EF46A12009C
:0A6D2600056A080EE76ED8900936E2
:106D300005360E50055C02E3056E092AE72EF7D7EB
:026D400012003F
:0E6D420000EE00F00F0EEE6AEA62FDD71200BE
:026D500012002F
:066D52000000000000003B
:086D580018101410140094023D
:026D6000A5028A
:0E6D6200000057FFFF0000FFFF000001015D71
:106D70000E00000000000000000000000000000005
:106D80000000000000000000000000000000000003
:106D900000000000000000000000000000000000F3
:106DA00000000000000000000000000000000000E3
:106DB00000000000000000000000000000000000D3
:0A6DC000000000FEFE28E0010101C2
:020000040030CA
:0100010006F8
:0100020018E5
:010003001AE2
:010005008179
:010006008178
:00000001FF
